:100000000C9407070C942F070C942F070C947A2854
:100010000C94B0280C948C280C942F070C942F0768
:100020000C942F070C94E9260C942F070C942F079F
:100030000C942F070C942F070C942F070C942F0768
:100040000C9447260C942F070C94B7260C949126F9
:100050000C942F070C942F070C942F070C942F0748
:100060000C945B270C942F074469657420312D3460
:1000700000436F6E6669726D203F00456E74657255
:100080000044656C617900536C65657000566F6C57
:1000900074616765004C6F772074682E004261744C
:1000A0007465727900436F6C6F720044656C697699
:1000B000657279004C69676874730054696D652FC7
:1000C000556E697400436F6E6669726D203F005211
:1000D000657365740056657273696F6E00524649A8
:1000E00044004469657434004469657433004469AC
:1000F000657432004469657431004669786564004E
:100100004D616E75616C004D6F64650047656E658D
:1001100072616C004C69676874203E20436F6C6F9D
:10012000727320004C69676874203E2044656C69D6
:100130007665727920282529004D656E75203E2050
:100140004C696768740054696D652F556E69742039
:100150003E2044696574340054696D652F556E699D
:1001600074203E2044696574330054696D652F55D1
:100170006E6974203E2044696574320054696D656F
:100180002F556E6974203E204469657431004D65B9
:100190006E75203E2054696D652F556E697400445C
:1001A0006174653A32302F30322F32303236005699
:1001B000657273696F6E3A322E302E3131004D6F99
:1001C0006465203E20466978650044696574203185
:1001D0002D34203E204469657434004469657420E0
:1001E000312D34203E2044696574330044696574C0
:1001F00020312D34203E2044696574320044696505
:100200007420312D34203E204469657431004D65E1
:100210006E75203E204469657420312D3400536C86
:10022000656570203E20456E74657200536C65658F
:1002300070203E2044656C6179004D656E75203EEE
:1002400020536C656570004D656E75203E20536CC3
:10025000656570004C6F772074682E203E20566FC5
:100260006C740042617474657279203E20566F6C24
:1002700074616765004D656E75203E20426174743F
:10028000657279004D656E75203E2042617474651B
:1002900072790047656E6572616C203E205265730D
:1002A00065740047656E6572616C203E204D6F6419
:1002B00065004D656E75203E2047656E6572616C08
:1002C000004D656E7500446C76640051747479005D
:1002D00073007300446965742031004469657420BB
:1002E0003400446965742033004469657420320029
:1002F00044696574203100446965742034004469A0
:100300006574203300446965742032004469657463
:1003100020310052464944004669786564004D61C9
:100320006E75616C00536F6C6964004C697175691E
:1003300064004E6F206D6F64756C65206465746534
:10034000637465642E00536541466F6F440000007E
:100350000000003E5B4F5B3E3E6B4F6B3E1C3E7CA5
:100360003E1C183C7E3C181C577D571C1C5E7F5E53
:100370001C00183C1800FFE7C3E7FF001824180012
:10038000FFE7DBE7FF30483A060E262979292640A9
:100390007F050507407F05253F5A3CE73C5A7F3ED5
:1003A0001C1C08081C1C3E7F14227F22145F5F0067
:1003B0005F5F06097F017F006689956A6060606003
:1003C0006094A2FFA29408047E040810207E2010EE
:1003D00008082A1C08081C2A08081E101010100CF7
:1003E0001E0C1E0C30383E3830060E3E0E06000045
:1003F00000000000005F00000007000700147F14E9
:100400007F14242A7F2A1223130864623649562057
:10041000500008070300001C2241000041221C007C
:100420002A1C7F1C2A08083E08080080703000083B
:1004300008080808000060600020100804023E510F
:1004400049453E00427F40007249494946214149A1
:100450004D331814127F1027454545393C4A494908
:100460003141211109073649494936464949291E72
:100470000000140000004034000000081422411461
:1004800014141414004122140802015909063E41B3
:100490005D594E7C1211127C7F494949363E4141DB
:1004A00041227F4141413E7F494949417F09090934
:1004B000013E414151737F0808087F00417F4100A0
:1004C0002040413F017F081422417F404040407F4F
:1004D000021C027F7F0408107F3E4141413E7F099C
:1004E0000909063E4151215E7F09192946264949DD
:1004F000493203017F01033F4040403F1F2040201D
:100500001F3F4038403F631408146303047804031A
:100510006159494D43007F414141020408102000C8
:100520004141417F04020102044040404040000339
:1005300007080020545478407F2844443838444405
:100540004428384444287F385454541800087E09FD
:100550000218A4A49C787F0804047800447D40001D
:100560002040403D007F1028440000417F40007C37
:10057000047804787C080404783844444438FC182F
:1005800024241818242418FC7C0804040848545413
:10059000542404043F44243C4040207C1C20402040
:1005A0001C3C4030403C44281028444C9090907CA7
:1005B0004464544C440008364100000077000000B9
:1005C0004136080002010204023C2623263C1EA1FB
:1005D000A161123A4040207A38545455592155555A
:1005E0007941225454784221555478402054557909
:1005F000400C1E527212395555555939545454599C
:1006000039555454580000457C410002457D420054
:1006100001457C407D1211127DF0282528F07C5484
:100620005545002054547C547C0A097F493249497D
:1006300049323A4444443A324A4848303A414121E6
:100640007A3A42402078009DA0A07D3D4242423D42
:100650003D4040403D3C24FF2424487E4943662BD6
:100660002FFC2F2BFF0929F620C0887E0903205478
:100670005479410000447D413048484A3238404076
:10068000227A007A0A0A727D0D19317D2629292FD6
:1006900028262929292630484D40203808080808EE
:1006A00008080808382F10C8ACBA2F102834FA00F0
:1006B000007B000008142A142222142A1408550072
:1006C000550055AA55AA55AAFF55FF55FF00000031
:1006D000FF00101010FF00141414FF001010FF0092
:1006E000FF1010F010F0141414FC001414F700FFA5
:1006F0000000FF00FF1414F404FC141417101F1062
:10070000101F101F1414141F00101010F000000010
:10071000001F101010101F10101010F0100000001B
:10072000FF101010101010101010FF10000000FF2C
:10073000140000FF00FF00001F10170000FC04F46D
:1007400014141710171414F404F40000FF00F71425
:10075000141414141414F700F714141417141010AC
:100760001F101F141414F4141010F010F000001FC8
:10077000101F0000001F14000000FC140000F01007
:10078000F01010FF10FF141414FF141010101F00AD
:10079000000000F010FFFFFFFFFFF0F0F0F0F0FFAF
:1007A000FFFF0000000000FFFF0F0F0F0F0F384486
:1007B000443844FC4A4A4A347E02020606027E025B
:1007C0007E0263554941633844443C04407E201E08
:1007D0002006027E020299A5E7A5991C2A492A1C37
:1007E0004C7201724C304A4D4D303048784830BC24
:1007F000625A463D3E494949007E0101017E2A2A4E
:100800002A2A2A44445F444440514A444040444ACE
:1008100051400000FF0103E080FF000008086B6BFF
:10082000083612362436060F090F06000018180085
:1008300000001010003040FF0101001F01011E00E8
:10084000191D1712003C3C3C3C0000000000000158
:1008500003070F1F3F7F0080C0E0F0F8FCFE574108
:10086000524E494E473A20436F6D6D756E69636114
:1008700074696F6E206661696C7572652C2069738E
:1008800020746865204D4652433532322070726FB5
:100890007065726C7920636F6E6E65637465643F1A
:1008A00000203D2028756E6B6E6F776E2900203D0D
:1008B00020636F756E74657266656974206368691C
:1008C0007000203D2076322E3000203D2076312EE3
:1008D0003000203D2076302E3000203D2028636CF3
:1008E0006F6E6529004669726D7761726520566585
:1008F0007273696F6E3A20307800DB40A4A62EAF89
:100900002000A1C8D300408DAED580A800006000B3
:1009100000000000000000000000000000E00000F7
:10092000000000000000000000000001E0000000E6
:100930000000000000000000000001F000000000C6
:1009400000000000000000000003F00000000000B4
:10095000000000000000000007F0000000000000A0
:100960000000000000000007F80000000000000088
:100970000000000000000FF800000003C0007E002F
:100980000001E0007F0FF800000003C000FE00003F
:1009900001E000FFEFF800000003C000FE000001CE
:1009A000E000FFFFF800000003C000F00000000FAF
:1009B000007FFE7FC0000003C000F00000000F00B9
:1009C0003FFE7FF83FF1FBCFFCFEF3BC3DEFE01FA5
:1009D000FE7FFF7FFBFFDFFEFEFFBC3DEFE01FC69B
:1009E000FFFF7FFBFFDFFEFEFFBC3DEFE00FE3C735
:1009F000FE787BC3DE1EF0FFBC3DEF0007FF87FCE7
:100A0000787BC3DE1EF0F83C3DEF0001FFFFF000F5
:100A10007BC3C01EF0F03C3DEF0001F37FE03FFBE5
:100A2000C3CFFEF0F03C3DEF0003E33F807FFBC30C
:100A3000DFFEF0F03C3DEF0007E73C00787BC3DED3
:100A40001EF0F03C3DEF0007FFBE00787BC3DE1ECA
:100A5000F0F03C3DEF0007FFFE00787BC3DE1EF0A8
:100A6000F03C3DEF000FFFFE007FFBFFDFFEF0F0EC
:100A70003FFDEFE00FFFFF007FFBFFDFFEF0F03FE9
:100A8000FDEFE00FF9FF003E79F9CF9EF0F01F3D3A
:100A9000E7E01FF1FF000000000000000000000080
:100AA000001F80FF007FFFFFFFFFFFFFFFFFFFE052
:100AB0001C007F007FFFFFFFFEB46D888D18E000F3
:100AC000001F007FFFFFFFFE95AD7DB577E00000C2
:100AD0000F007FFFFFFFFEA5AD9D8D19E000000612
:100AE000007FFFFFFFFEB5ADEDB57EE0000000002A
:100AF00000018000000000000000000003800000F2
:100B00000000000000000007C0000000000000001E
:100B1000000007C00000000000000000000FC0003F
:100B200000000000000000001FE0000000000000C6
:100B30000000001FE00000000000000000003FE097
:100B40000000000000000000003FF0000000000076
:100B5000000000007FF0000000000000001FF87F90
:100B6000F0000000000000003FFE7FF000000000E9
:100B70000000003FFF7FF0000000000000001FFFAA
:100B8000FBE0000000000000000FFFF9FFC00000C4
:100B9000000000000FFFF9FFF80000000000000750
:100BA000FFF1FFFF00000000000003FC73FFFF8067
:100BB000000000000001FE3FFFFF80000000000079
:100BC00000FF1E0FFF000000000000007FFE1FFC62
:100BD000000000000000003FFFFFF80000000000E0
:100BE00000000FDFFFE0000000000000001F19FF01
:100BF000C0000000000000003F3CFF0000000000BB
:100C00000000007E7CF800000000000000007FFE75
:100C10007C0000000000000000FFFFFC000000005E
:100C200000000000FFFFFE0000000000000000FFC9
:100C3000FFFE0000000000000001FFEFFE000000CA
:100C40000000000001FFCFFE0000000000000003D4
:100C5000FF07FE0000000000000003FC07FE00008C
:100C6000000000000003F003FE0000000000000090
:100C7000018000FE000000000000000000007E0077
:100C80000000000000000000003E00000000000026
:100C9000000000000C000000000000078000FC00C5
:100CA0000003C0000000078001FC000003C000003A
:100CB00000078001FC000003C0000000078001E085
:100CC0000000001E000000078001E00000001E0080
:100CD0007FE3F79FF9FDE7787BDFC0FFF7FFBFFDFC
:100CE000FDFF787BDFC0FFF7FFBFFDFDFF787BDFF7
:100CF000C0F0F787BC3DE1FF787BDE00F0F787BCF2
:100D00003DE1F0787BDE0000F787803DE1E0787B15
:100D1000DE007FF7879FFDE1E0787BDE00FFF7874D
:100D2000BFFDE1E0787BDE00F0F787BC3DE1E078D5
:100D30007BDE00F0F787BC3DE1E0787BDE00F0F77A
:100D400087BC3DE1E0787BDE00FFF7FFBFFDE1E01F
:100D50007FFBDFC0FFF7FFBFFDE1E07FFBDFC07C73
:100D6000F3F39F3DE1E03E7BCFC0000000000000B8
:100D70000000000000FFFFFFFFFFFFFFFFFFFFC0BD
:100D8000FFFFFFFFFD68DB111A31C0FFFFFFFFFD12
:100D90002B5AFB6AEFC0FFFFFFFFFD4B5B3B1A3393
:100DA000C0FFFFFFFFFD6B5BDB6AFDC000000000C2
:100DB000240027002A0000000000250028002B0046
:100DC0000000000023002600290004040404040499
:100DD00004040202020202020303030303030102EA
:100DE00004081020408001020408102001020408B9
:100DF00010200000000800020100000304070000AA
:100E00000000000000002200FF21D4282635112414
:100E10001FBECFEFD8E0DEBFCDBF24E0A8EFB1E02A
:100E200001C01D92A130B207E1F711E0A0E0B1E0EE
:100E3000ECE0F5E702C005900D92A83FB107D9F7A5
:100E400017E0C6E0D7E004C02197FE010E94613898
:100E5000C530D107C9F70E9465290C94793A0C94E2
:100E600000000895833081F028F4813099F08230B9
:100E7000A9F008958730A9F08830C9F08430B1F422
:100E8000809180008F7D03C0809180008F77809358
:100E90008000089584B58F7784BD089584B58F7DD3
:100EA000FBCF8091B0008F778093B0000895809140
:100EB000B0008F7DF9CFCF93DF93282F30E0F90179
:100EC000EE50F24F8491F901E252F24FD491F901C0
:100ED000E653F24FC491CC23A1F081110E94320756
:100EE000EC2FF0E0EE0FFF1FE054F24FA591B4910C
:100EF000EC91ED2381E090E009F480E0DF91CF9167
:100F0000089580E090E0FACF1F93CF93DF93282FCE
:100F100030E0F901EE50F24F8491F901E252F24FC4
:100F2000D491F901E653F24FC491CC23A9F0162FC6
:100F300081110E943207EC2FF0E0EE0FFF1FEA5400
:100F4000F24FA591B4918FB7F894EC91111108C0AC
:100F5000D095DE23DC938FBFDF91CF911F91089551
:100F6000DE2BF8CFCF93DF9390E0FC01E252F24FFB
:100F700024918653924FFC0184918823D1F090E014
:100F8000880F991FFC01E455F24FA591B491FC0123
:100F9000EA54F24FC591D49161110EC09FB7F894F5
:100FA0008C91E22FE0958E238C932881E223E883B5
:100FB0009FBFDF91CF9108958FB7F894EC91E22B0A
:100FC000EC938FBFF6CF1F93CF93DF93182FEB01D6
:100FD00061E00E94B207209739F460E0812FDF9131
:100FE000CF911F910C948407CF3FD10511F461E09C
:100FF000F5CFE12FF0E0EE50F24FE491E33031F124
:1010000040F4E130B1F0E230E1F0C038D1057CF7D6
:10101000E4CFE73029F1E83059F1E430B1F78091BD
:101020008000806280938000D0938B00C0938A0000
:1010300004C084B5806884BDC7BDDF91CF911F9186
:10104000089584B5806284BDC8BDF7CF80918000CB
:10105000806880938000D0938900C0938800EDCF92
:101060008091B00080688093B000C093B300E5CF5A
:101070008091B00080628093B000C093B400DDCF57
:101080008E50806480937C0080917A00806480938D
:101090007A0080917A0086FDFCCF80917800909153
:1010A000790008953FB7F8948091F6029091F70285
:1010B000A091F802B091F90226B5A89B05C02F3F78
:1010C00019F00196A11DB11D3FBFBA2FA92F982F6E
:1010D0008827BC01CD01620F711D811D911D42E069
:1010E000660F771F881F991F4A95D1F708958F9231
:1010F0009F92AF92BF92CF92DF92EF92FF924B01FD
:101100005C010E9452086B017C010E9452086C191C
:101110007D098E099F09683E734081059105A8F3FA
:1011200021E0821A9108A108B10888EEC80E83E078
:10113000D81EE11CF11C81149104A104B10429F70B
:10114000FF90EF90DF90CF90BF90AF909F908F90E7
:1011500008952FB7F8946091F2027091F302809194
:10116000F4029091F5022FBF08950895089508950F
:10117000EF92FF920F931F93CF93DF938C017B012C
:10118000D0E0C0E0F701EC0FFD1F6491662361F031
:10119000D801ED91FC910190F081E02DC8010995F5
:1011A000892B11F02196EECFCE01DF91CF911F91C7
:1011B0000F91FF90EF900895AF92BF92CF92DF9280
:1011C000EF92FF920F931F93CF93DF936C017B01FC
:1011D0008B01040F151FEB015E01AE18BF08C0178D
:1011E000D10759F06991D601ED91FC910190F08100
:1011F000E02DC6010995892B79F7C501DF91CF91C3
:101200001F910F91FF90EF90DF90CF90BF90AF9024
:101210000895FC01538D448D252F30E0842F90E0FC
:10122000821B930B541710F0CF96089501970895E1
:10123000FC01918D828D981761F0A28DAE0FBF2FAA
:10124000B11D5D968C91928D9F5F9F73928F90E000
:1012500008958FEF9FEF0895FC01918D828D98176F
:1012600031F0828DE80FF11D858D90E008958FEFAC
:101270009FEF0895FC01918D228D892F90E0805C75
:101280009F4F821B91098F73992708958EEF92E0EB
:101290000E943A0921E0892B09F420E0822F089569
:1012A00080E090E0892B29F00E94460981110C947E
:1012B00000000895FC01A48DA80FB92FB11DA35AF9
:1012C000BF4F2C91848D90E001968F739927848F66
:1012D000A689B7892C93A089B1898C918370806489
:1012E0008C93938D848D981306C00288F389E02D2A
:1012F00080818F7D80830895EF92FF920F931F93DB
:10130000CF93DF93EC0181E0888F9B8D8C8D9813B8
:101310001AC0E889F989808185FF15C09FB7F894C4
:10132000EE89FF896083E889F98980818370806410
:1013300080839FBF81E090E0DF91CF911F910F915B
:10134000FF90EF900895F62E0B8D10E00F5F1F4F6A
:101350000F731127E02E8C8D8E110CC00FB607FC79
:10136000FACFE889F989808185FFF5CFCE010E9407
:101370005A09F1CFEB8DEC0FFD2FF11DE35AFF4F12
:10138000F0829FB7F8940B8FEA89FB898081806295
:10139000CFCFCF93DF93EC01888D8823B9F0AA8952
:1013A000BB89E889F9898C9185FD03C0808186FD20
:1013B0000DC00FB607FCF7CF8C9185FFF2CF80816F
:1013C00085FFEDCFCE010E945A09E9CFDF91CF9181
:1013D00008958EEF92E00E94C909EEEFF2E0A28933
:1013E000B3898C918F7E8C93A289B3898C91877FEE
:1013F0008C93A289B3898C918F778C93A289B389BE
:101400008C918F7D8C93828D818F0895BC016E5F4E
:101410007F4FDC01ED91FC910190F081E02D40E0E7
:10142000099591E0811190E0892F0895EF92FF9244
:101430000F931F93CF93DF93EC01EC80FD806E152B
:101440007F050CF070C057FF04C0240F351F50E01B
:1014500040E08E819F81FA01E20FF31F8E179F07F4
:101460001CF49C01241B350B121613060CF05BC0F8
:10147000922F842F8695869586958E9DD0018F9D7F
:10148000B00D11246A0F7B1FAF8DB8A1A60FB71F37
:10149000477049F188E0841B482F682F70E0FB01FA
:1014A000EA5AF74FE491281708F063C0621B7109EC
:1014B0002FEF30E002C0359527956A95E2F7E223D9
:1014C0000130110539F0B0F10230110561F58C9150
:1014D000E82702C08C91E82BEC93941720F12C8123
:1014E0003D81A20FB31FE92FE41BE83078F00230F2
:1014F000110521F58E2F9C9190959C932C813D8117
:10150000A20FB31F88508830B0F7E770EE2359F070
:10151000F0E0E25BF74FE49101301105F9F010F1D2
:101520000230110519F1DF91CF911F910F91FF90BA
:10153000EF900895E0958C91E823CECF81E00115DE
:10154000110509F480E081959E2F8C932C813D81BB
:10155000A20FB31F98509830C0F7D7CF8C91E82BCB
:10156000EC93E1CFE0958C91E823FACF8C91E827BA
:10157000F7CF0130110509F4ADCFE0F202301105CB
:1015800009F4A5CFAE0DBF1DAECF0F931F93CF9320
:10159000DF9377FF04C0260F371F70E060E0DC01A7
:1015A0001496CD91DC91FB01E20FF31FCE17DF07FC
:1015B0001CF49E01261B370B121613064CF5FA017C
:1015C00057FD3796A3E0F595E795AA95E1F7EC9FCF
:1015D000D001ED9FB00DFC9FB00D11246A0F7B1F51
:1015E000DC015F96ED91FC91E60FF71F47705527E0
:1015F00081E090E001C0880F4A95EAF7482F01305A
:10160000110559F0A8F02E0F3F1F02301105E1F02F
:10161000DF91CF911F910F9108952E0F3F1FE21779
:10162000F307B1F38191DF011197842B8C93F7CFEE
:1016300080952E0F3F1FE217F30751F39191DF01C1
:10164000119798239C93F7CFE217F30709F3819141
:10165000DF01119784278C93F7CF0F931F93FA0123
:10166000DC0156964C9156974230E9F04330A1F197
:10167000413061F514964D915C91DA01AE1BBF0BC0
:10168000FD01E21BF30B77FD0BC0DC0116964D91BB
:101690005C916417750724F4AB01BF010E94C50A71
:1016A0001F910F91089514964D915C91DA01A61B3C
:1016B000B70BBD0161507109DC0116964D915C912B
:1016C000DA01AE1BBF0BFD01E21BF30B77FDE8CF88
:1016D000AF010E94160AE4CF16964D915C91DA0193
:1016E000A61BB70BBD0161507109CDCF0F931F939E
:1016F000FA01DC0156964C9156974230A9F04330DE
:1017000091F1413019F514964D915C91DA01AE1BBF
:10171000BF0BFD013197F7FD04C0AB01BF010E9473
:10172000160A1F910F91089514964D915C91DA015C
:10173000A61BB70BBD01DC0116964D915C91DA0139
:10174000AE1BBF0BFD013197621B730BF7FDE9CF99
:10175000DC0116964D915C91E417F50714F7AF0183
:101760000E94C50ADECF16964D915C91DA01A61B48
:10177000B70BBD01621B730BCECFFC0177FD64C0BC
:1017800080859185681779070CF05EC057FD5CC0B5
:1017900082859385481759070CF056C08689823098
:1017A000B1F0833029F1813041F484819581841B2B
:1017B000950BAB01BC01615071092130310509F174
:1017C00008F443C02230310509F463C008958481D0
:1017D0009581DC01A61BB70BBD01615071098681A3
:1017E0009781DC01A41BB50BAD0141505109E5CF38
:1017F00086819781861B970BBA01AC014150510934
:10180000DCCFCA0157FD0796A3E095958795AA9569
:10181000E1F7A481B5818A9F90018B9F300D9A9F3B
:10182000300D1124620F731F078CF0A1E02DE60F1D
:10183000F71F4770552721E030E001C0220F4A957D
:10184000EAF78081822B80830895CA0157FD0796AD
:1018500033E0959587953A95E1F7A481B5818A9F04
:1018600090018B9F300D9A9F300D1124620F731FD2
:10187000078CF0A1E02DE60FF71F4770552781E098
:1018800090E001C0880F4A95EAF7809590818923FE
:10189000DACFCA0157FD079623E0959587952A95DB
:1018A000E1F7A481B5818A9F90018B9F300D9A9FAB
:1018B000300D1124620F731F078CF0A1E02DE60F8D
:1018C000F71F4770552721E030E001C0220F4A95ED
:1018D000EAF780818227B7CF8091AA02882361F03E
:1018E0009FB7F8942091AA028091A902213019F49F
:1018F0008DBB9FBF08958FBF08958EBD00000DB4AE
:1019000007FEFDCF8EB508952091AA02222361F033
:101910002FB7F8943091AA02313049F43DB3309397
:10192000A9023DB33DBB2FBF8CBD9DBD0895209343
:10193000A902FACFDF92EF92FF920F931F93CF93FA
:10194000DF937C01062FD42E152F80E590E00E94B6
:10195000840C60E0F70186850E94840782E10E9482
:101960007D0CCD2DD12F0C0F1D2F111DC017D107B0
:1019700021F089910E947D0CF9CF61E0F701868505
:101980000E948407DF91CF911F910F91FF90EF90FC
:10199000DF900C946C0C1F93CF93DF93EC01162F08
:1019A00080E590E00E94840C60E08E850E948407B0
:1019B000812F80680E947D0C80E00E947D0C182F92
:1019C00061E08E850E9484070E946C0C812FDF915C
:1019D000CF911F9108950F931F93CF93DF93EC0145
:1019E000062F142F80E590E00E94840C60E08E8525
:1019F0000E948407802F0E947D0C812F0E947D0C05
:101A000061E08E850E948407DF91CF911F910F9135
:101A10000C946C0CCF92DF92EF92FF920F931F9376
:101A2000CF93DF93EC016B01F42E890140E062E07B
:101A30000E94EB0C44E06AE0CE010E94EB0C40E80F
:101A400064E1CE010E94EB0CA6016F2DCE010E9435
:101A50009A0C43E062E0CE010E94EB0C0E94A908C0
:101A60006B017C0129E5C20ED11CE11CF11C6AE06E
:101A7000CE010E94CB0C82FF1BC040E062E0CE0191
:101A80000E94EB0C64E4CE010E94CB0CF801808331
:101A900062E4CE010E94CB0CF801818380E0DF91EB
:101AA000CF911F910F91FF90EF90DF90CF9008950D
:101AB0000E94A9086C157D058E059F05C0F283E084
:101AC000EECF2F923F924F925F926F927F928F92C2
:101AD0009F92AF92CF92DF92EF92FF920F931F935C
:101AE000CF93DF9300D0CDB7DEB74C012B01D42EBE
:101AF000390180E0E114F10411F0F70180813C2C00
:101B0000329490EF3922380E40E062E0C4010E9426
:101B1000EB0C4FE768E0C4010E94EB0C40E864E185
:101B2000C4010E94EB0CA2016D2DC4010E949A0C0D
:101B3000432D6AE1C4010E94EB0C4CE062E0C40159
:101B40000E94EB0C6AE1C4010E94CB0C482F406854
:101B50006AE1C4010E94EB0C0E94A9081B012C0140
:101B6000F4E22F0E311C411C511C68E0C4010E949C
:101B7000CB0C982F907309F0B9C080FF15C083E09B
:101B80000F900F90DF91CF911F910F91FF90EF90E9
:101B9000DF90CF90AF909F908F907F906F905F90ED
:101BA0004F903F902F9008950E94A90862157305E9
:101BB00084059505D0F2E3CF6114710409F46BC07C
:101BC0000115110509F467C064E1C4010E94CB0C42
:101BD000382EF8018081831508F482C030823320CA
:101BE000F1F180E590E00E94840C60E0F4018685CC
:101BF0000E9484073A9482E90E947D0CCC20B1F0C7
:101C00008FEF90E09C0102C0220F331FCA94E2F7CD
:101C1000690182E90E947D0C9C2D9095F301208141
:101C200092238C21982B9083CC24C39423014C0CB9
:101C3000511CC31440F482E90E947D0CF20181938F
:101C40002F01C394F6CF80E00E947D0CF2018083C7
:101C500061E0F40186850E9484070E946C0C68E1B3
:101C6000C4010E94CB0C8770E114F10411F0F7015C
:101C7000808323FC37C061147104B1F10115110593
:101C800099F1AA2089F1F8014081413031F4843082
:101C900029F58FEF75CF80E0ECCF4230F8F081115D
:101CA0001DC042509E012F5F3F4FB301C4010E94EF
:101CB0000A0D811165CFF8019081690E711CF30145
:101CC000329720819981291309C0F1E06F1A7108B8
:101CD000F30120819A81291709F452CF87E050CF70
:101CE00084E04ECF82E04CCF80E04ACF6CE0C4016C
:101CF0000E94CB0C282E837109F45ECF81E040CF87
:101D00000F931F93CF93DF938C01D62FC42F0E9484
:101D1000CB0CC0954C2F48236D2FC801DF91CF917C
:101D20001F910F910C94EB0C8F929F92AF92CF92D8
:101D3000EF92FF920F931F93CF93DF9300D000D0C9
:101D40001F92CDB7DEB74C0182E08D8340E064E2A4
:101D5000C4010E94EB0C40E066E2C4010E94EB0C5F
:101D600046E268E4C4010E94EB0C86E28B838D811D
:101D70008230B0F140E86CE1C4010E94800E87E03F
:101D80008C83A12CC12CCE0104967C018E010B5FAB
:101D90001F4F9E012F5F3F4F41E0BE016D5F7F4FA0
:101DA000C4010E94610D982F811117C08D8182306E
:101DB000B9F48C81811114C081E00F900F900F90C5
:101DC0000F900F90DF91CF911F910F91FF90EF90A7
:101DD000CF90AF909F908F90089581E0923069F3FB
:101DE00080E0EBCF2F923F924F925F926F927F9263
:101DF0008F929F92AF92BF92CF92DF92EF92FF921B
:101E00000F931F93CF93DF93CDB7DEB72D970FB608
:101E1000F894DEBF0FBECDBF16E0413508F045C1D6
:101E2000342E4B013C0140E86CE10E94800E83E9B6
:101E30008983332029F081E0F4019081953008F402
:101E400080E022242394B12C9B2D990F990F990F98
:101E5000D32CD91AD7FCD12C32E0882319F098E87A
:101E60009B8333E021E09D2D977009F420E09D2DA8
:101E7000959595959595290FC9F094E0811193E07A
:101E8000291708F4922FEB2DF0E03196E80DF91D9B
:101E9000232F4191A1E0B0E0AC0FBD1FA20FB11DF7
:101EA0004C932F5F422F431B491798F3882311F05F
:101EB000F8E0DF0E8FE18D150CF082C090E79A8379
:101EC0008B819C8189279D8189279E8189278F838A
:101ED0009E01285F3F4F47E0BE016F5F7F4FC30108
:101EE0000E940A0D182F8111E0C01A86E3E0EB87EB
:101EF000DC86CE0107962C0199E09D87CA844C2D83
:101F00004295407F4C0D6AE1C3010E94EB0CA12C6D
:101F1000CE010A967C018E01055F1F4F92014D850F
:101F2000BE016F5F7F4FC3010E94610D182F823089
:101F300009F065C06CE1C3010E94CB0C85FDB5C002
:101F40008F7109F480E2282F30E04D2DDD0C550B08
:101F5000421753070CF09DC0D82EE82FE595E59564
:101F6000E595EF5F982F977081E009F480E0E80F26
:101F700081E090E08C0F9D1F8E0F911DFC01215080
:101F800031092770332781E090E002C0880F991F44
:101F90002A95E2F79C018081822B80838BCF85E993
:101FA0008983332031F081E0F4019081983008F08A
:101FB0004BCF80E049CF87E9898326E0B22EF9CF65
:101FC0009D2D97709A878D2D8595859585958E5F2A
:101FD000282F2295207F290F2A8321E0911101C00B
:101FE00020E0280F2D8744244394512C4C0E5D1E75
:101FF000480E511CE9E0E81BEB87DC867FCF81119E
:1020000054C080E2D82E9C8590320CF457CF8B813F
:10201000883809F040C083E093E0EB2DF0E0319682
:10202000E80DF91D980FA1E0B0E0AC0FBD1FA80F9F
:10203000B11D2C9121938F5F8913F5CFBB84E3E011
:10204000BE124DC08A8581114AC09E012D5F3F4F4F
:1020500041E0B201C3010E940A0D182F811125C071
:102060009B81F201818198133CC09C8182819813ED
:1020700038C0808182FF12C02394F2E02F1609F449
:102080008ECF83E0281609F496CF91E0291609F443
:10209000CECE15E00AC082E094E0BFCFF401838782
:1020A000822D880F820D8F5F8083812F2D960FB632
:1020B000F894DEBF0FBECDBFDF91CF911F910F917E
:1020C000FF90EF90DF90CF90BF90AF909F908F9058
:1020D0007F906F905F904F903F902F90089511E008
:1020E000E4CF17E0E2CF0895FC016370668B848132
:1020F000958126813781613039F0633029F09187ED
:102100008087338722870895318720879387828746
:1021100008952F923F924F925F926F927F928F928B
:102120009F92AF92BF92CF92DF92EF92FF920F9366
:102130001F93CF93DF93CDB7DEB76A970FB6F894AE
:10214000DEBF0FBECDBF9A8F898F7A8369834A0124
:10215000D22E18870F833701BC2CDC0159962D91A4
:102160003C915A972115310509F015C118968D91AA
:102170009C911997681779070CF0D7C11A968D9121
:102180009C91481759070CF0D0C14C2C512CB6E04B
:10219000CB9E600D711D11247C876B871616170668
:1021A0000CF0C3C1EA2DF0E0FA87E98793E0EE0F67
:1021B000FF1F9A95E1F7F88BEF87CF01840F951FEA
:1021C000181619060CF0B1C1A98DBA8D58968C91CC
:1021D000811104C0BFEABD1508F4D394A98DBA8D4E
:1021E000ED91FC9111970284F385E02DCD010995C5
:1021F000B5E0DB9EC0011124E981FA81FC83EB8309
:10220000312C212C9C01225B3C4F388F2F8B4A2D87
:1022100050E05E8B4D8BEF89F88DE20DF31D4491FC
:102220009E828D82D12CC12C69817A81620D731DB1
:102230007A8B698B842F90E09C8B8B8BE98DFA8D48
:10224000A081B18140FF82C0F1E0BF126FC0AF1228
:102250006DC01C96ED91FC912F813885A4014C0D29
:102260005D1D69897A89898D9A8D0995EB89FC892B
:10227000F595E7954E2F5FEFC51AD50A6D817E81E2
:102280008D899E89680F791F7E836D8398E0C916BA
:10229000D10481F6AFEF2A1A3A0AEB81FC81E40DF2
:1022A000F51DFC83EB83F5E02F16310409F0B3CF65
:1022B0002F81388526153705B9F0A98DBA8DED9196
:1022C000FC91B1E0BB1257C0AB1255C069817A8155
:1022D0006B5F7F4F0088F189E02D830128E030E0BB
:1022E000A401898D9A8D0995A98DBA8DED91FC91E6
:1022F00011970688F789E02DCD016A960FB6F894FC
:10230000DEBF0FBECDBFDF91CF911F910F91FF9028
:10231000EF90DF90CF90BF90AF909F908F907F9085
:102320006F905F904F903F902F9009941E96ED9183
:10233000FC91EF80F88409851A8592014D815E81B8
:102340006B817C81898D9A8D099590CF2F813885FD
:102350002615370509F48ACF31E0B31207C0A3125E
:1023600005C01C96ED91FC91930178CF1E96ED91DE
:10237000FC917301E0CF6B857C8564197509068437
:10238000F785E02D73010F8518899201A401898DCD
:102390009A8D0995A9CFF901349694913297459178
:1023A0005491D91AB7E0DB9E400D511D1124F9015B
:1023B000259134913C8B2B8BFA0125903490FA01B6
:1023C0003296749031963491398B3296649031966E
:1023D000449041E04C1518F04A1508F07FC0662D76
:1023E000062C000C770B7C836B83842D042C000C53
:1023F000990B9E838D83A98DBA8DED91FC911197D8
:102400000284F385E02DCD010995512CD12CC12CEE
:10241000EA2DF0E0FA87E9872B2D30E03C872B8707
:10242000A401440D511D47FC5A95588F4F8B69816B
:102430007A81660D711D67FC7A957E876D87798933
:10244000C71608F051CF2C2D30E04D815E81420F30
:10245000531FA985BA854A9FC0014B9F900D5A9F73
:10246000900D1124FC01E80DF91DF88BEF87852DE7
:10247000612C4F89588D420F531F5E8B4D8B671413
:1024800008F050C044244394480E877041F4C101C1
:102490000196EB89FC89E20DF31DD4901C01D7FE57
:1024A00019C0A98DBA8DED91FC91662D70E0B1E057
:1024B000BB1219C0AB1217C02D853E85620F731F6A
:1024C0000484F585E02D2F8138854D895E89898DBD
:1024D0009A8D0995DD0C6394842DD1CF1E821D82C7
:1024E0001C821B8288CF4B815C81640F751FAB857A
:1024F000BC856A9FC0016B9F900D7A9F900D11243F
:1025000069817A81680F791F0684F785E02DEF8055
:10251000F88409851A859D014F855889898D9A8D82
:102520000995D8CF570CC3948ACF6A960FB6F89402
:10253000DEBF0FBECDBFDF91CF911F910F91FF90F6
:10254000EF90DF90CF90BF90AF909F908F907F9053
:102550006F905F904F903F902F9008958F929F9231
:10256000AF92CF92EF92FF920F931F93CF93DF938F
:10257000EC01262F898D9A8D009709F051C06A30A1
:10258000D1F41D861C868D8948E0849F900111241A
:102590008E859F85820F931F9F878E8781E090E0B5
:1025A000DF91CF911F910F91FF90EF90CF90AF905F
:1025B0009F908F9008956D3089F3CC88AD888F8976
:1025C0008823C1F08C859D8536E0C39E800D911DCA
:1025D0001124488559854817590764F44E855F854D
:1025E0001D861C8638E0A39EC0011124840F951F10
:1025F0009F878E87EA88FB88088919894E855F85C1
:102600006C857D85CE010E9489102C898C859D85E5
:1026100046E0249F800D911D11249D878C87BECF9D
:102620006A3069F41D861C86FC013896E4912D8978
:102630008E859F85E29F800D911D1124ADCF6D3059
:1026400009F4ACCFFC0134963491631708F4A6CF9B
:102650003296E491E61708F4A1CFFC0132968590FA
:102660009490462F431B342F47E0349F800C911CDD
:102670001124F401329634913196E4913323A9F177
:10268000EE2399F1CC88F4013596E491AD884F8919
:10269000442301F10E2E000CFF0BE30FF11DCE9E23
:1026A000A001CF9E500D11246C857D85460F571FCC
:1026B00068857985641775076CF44E855F851D867E
:1026C0001C86FC013896E491AE9E400D511D1124EC
:1026D0005F874E87EA88FB88088919894E855F8560
:1026E0006C857D85CE010E948910F4013496E491B9
:1026F0002C898C859D85E29F800D911D11248DCFA5
:102700006F927F928F929F92AF92BF92CF92DF9201
:10271000EF92FF920F931F93CF93DF93EC016B0126
:102720005A0139014801E881F9810284F385E02DDD
:102730000995E881F9810288F389E02D87019301E9
:10274000A501B601CE010995A501480D591D4150BD
:102750005109E881F9810288F389E02D9301B601DE
:10276000CE010995E881F9810088F189E02D940175
:10277000A501B601CE010995C60CD71CB601615062
:102780007109E881F9810088F189E02D9401A501A2
:10279000CE010995E881F9810688F789E02DCE01FF
:1027A000DF91CF911F910F91FF90EF90DF90CF902D
:1027B000BF90AF909F908F907F906F9009946F9291
:1027C0007F928F929F92AF92BF92CF92DF92EF92C1
:1027D000FF920F931F93CF93DF935C01EB016A018C
:1027E000490138018701DC01ED91FC916217730703
:1027F00019F5641675062CF0962D872D3A01C92E11
:10280000D82E9601261937092F5F3F4F048CF58D7E
:10281000E02DA301BE01C5010995DF91CF911F9164
:102820000F91FF90EF90DF90CF90BF90AF909F906F
:102830008F907F906F9008954615570591F4261755
:10284000370724F0892D4B01C22FD82F9E0128195C
:1028500039092F5F3F4F068CF78DE02DA601B4019B
:10286000DACF0284F385E02D0995D501ED91FC9135
:102870000488F589E02D83019401A601BE01C501FC
:102880000995D501ED91FC910688F789E02DC501E8
:10289000DF91CF911F910F91FF90EF90DF90CF903C
:1028A000BF90AF909F908F907F906F900994EF9220
:1028B000FF920F931F93DC011A960D911C911B97A9
:1028C00018962D913C911997ED91FC9100A0F1A1E2
:1028D000E02D7B0150E040E070E060E009951F9141
:1028E0000F91FF90EF9008954F925F926F927F92B9
:1028F0008F929F92AF92BF92CF92DF92EF92FF9210
:102900000F931F93CF93DF936C012B015A01390171
:102910004801DC01ED91FC910284F385E02D0995DD
:10292000E201640C751CD601ED91FC91C615D7052A
:102930005CF40088F189E02D87019401A501BE01B6
:10294000C60109952196EFCF0688F789E02DC601CB
:10295000DF91CF911F910F91FF90EF90DF90CF907B
:10296000BF90AF909F908F907F906F905F904F90AF
:1029700009948F929F92AF92BF92CF92DF92EF9283
:10298000FF920F931F93CF93DF93EC015B014A01FA
:102990006901E881F9810284F385E02D09959501AB
:1029A0002C0D3D1D21503109E881F9810488F589FC
:1029B000E02D78018401A401B501CE010995E881DB
:1029C000F9810688F789E02DCE01DF91CF911F9123
:1029D0000F91FF90EF90DF90CF90BF90AF909F90BE
:1029E0008F9009948F929F92AF92BF92CF92DF9275
:1029F000EF92FF920F931F93CF93DF93EC015B0154
:102A00004A0169017801E881F9810284F385E02DAA
:102A10000995C80CD91C860101501109E881F9817A
:102A20000488F589E02D9501A401B501CE01099531
:102A3000E881F9810688F789E02DCE01DF91CF91F9
:102A40001F910F91FF90EF90DF90CF90BF90AF90CC
:102A50009F908F900994EF92FF920F931F93DC0148
:102A6000ED91FC9100A0F1A1E02D09951F910F912E
:102A7000FF90EF9008950F931F93DC01ED91FC916F
:102A8000068CF78DE02D09951F910F9108950F93F6
:102A90001F93DC01ED91FC91048CF58DE02D0995DF
:102AA0001F910F910895DC01ED91FC910084F18557
:102AB000E02D09943F924F925F926F927F928F9296
:102AC0009F92AF92BF92CF92DF92EF92FF920F93BD
:102AD0001F93CF93DF935C017B014A0169013901A8
:102AE00087E0680E711C93E0759467949A95E1F7FE
:102AF0002B01400E511E10E000E0312CD0E0C0E070
:102B0000CE0187709927330C892B59F4FE0183E09D
:102B1000F595E7958A95E1F7E00FF11FE80DF91DAE
:102B2000349037FE0AC021E030E0A701B5016C0FF8
:102B30007D1F87EB93E00E9453152196CC16DD068E
:102B4000F9F68FEFE81AF80A060D171DE414F504DC
:102B5000A9F6DF91CF911F910F91FF90EF90DF9039
:102B6000CF90BF90AF909F908F907F906F905F902D
:102B70004F903F9008952F923F924F925F926F92A5
:102B80007F928F929F92AF92BF92CF92DF92EF92FD
:102B9000FF920F931F93CF93DF9300D000D000D00C
:102BA000CDB7DEB73C016A013E832D83FC82EB8208
:102BB0005801A41AB50AB7FE03C0B194A194B10894
:102BC0008D809E80861A970A97FE03C09194819407
:102BD00091088A149B045CF0902F812F0D811E8137
:102BE0009D838E839C2D8D2D6B01692F782F0C1565
:102BF0001D055CF09D818E817E836D83692F782F0A
:102C0000902F812F8601C92ED82E1601201A310A45
:102C10002B012D813E81421A530A57FE03C0519465
:102C200041945108710137FE03C03FEFE31AF30AE4
:102C3000F594E7948D819E81861797075CF5A1E056
:102C4000B0E0BA83A983C016D1064CF1D301ED914F
:102C5000FC910484F585E02D2B813C81A8016D81D8
:102C60007E818A149B041CF04D815E81B801C301F2
:102C70000995E418F508F7FE0AC02D813E81898187
:102C80009A81280F391F3E832D83E20CF31C0F5FBE
:102C90001F4FD9CF2FEF3FEF3A832983D4CF26960A
:102CA0000FB6F894DEBF0FBECDBFDF91CF911F915D
:102CB0000F91FF90EF90DF90CF90BF90AF909F90DB
:102CC0008F907F906F905F904F903F902F900895DE
:102CD00020915F02260F3327331F21323105ECF498
:102CE00020918302FC0190E080E0243069F082E0D2
:102CF0000895A0915F022191AC01415C5D4FA40F4A
:102D0000B52FB11D2C930196861798F380915F0221
:102D1000680F60935F0280E0089581E00895ECEB16
:102D2000F0E080818A7B808360E082E10E948407FA
:102D300060E083E10C9484071092830281E0809329
:102D400085021092840261E082E10E94840761E0C2
:102D500083E10E948407E9EBF0E080818E7F80832D
:102D600080818D7F808388E48093B80085E48093A0
:102D7000BC000895CF93DF9391E090933E028823A7
:102D800061F0C091B800D091BA000E948F160E94E5
:102D90009C16D093BA00C093B800DF91CF910895EC
:102DA000E091BD028091BC02E81730F4F0E0E75EEC
:102DB000FD4F808190E008958FEF9FEF08959091EF
:102DC000BD028091BC022FEF3FEF981748F4E92F26
:102DD000F0E0E75EFD4F208130E09F5F9093BD0201
:102DE000C90108958091BC029091BD02891B990B85
:102DF0000895CF92DF92EF92FF920F931F93CF939C
:102E0000DF937C01CB018A012091FD02222389F00E
:102E1000EB016B01C40ED51ECC15DD0569F069917F
:102E2000D701ED91FC910190F081E02DC70109954A
:102E3000F3CF642F0E946816C801DF91CF911F91D4
:102E40000F91FF90EF90DF90CF900895CF93DF9395
:102E50001F92CDB7DEB769832091FD022223F9F0DE
:102E60002091FA02203258F021E030E0FC01338357
:102E7000228390E080E00F90DF91CF9108958091C0
:102E8000FB02E82FF0E0E750FE4F998190838F5FBF
:102E90008093FB028093FA0281E090E0ECCF61E046
:102EA000CE0101960E946816F7CFCF92DF92EF9283
:102EB000FF920F931F93CF93DF93D091FA0281E09B
:102EC000D13208F09CC0C091FC020E9452086B01F4
:102ED0007C018091830281116CC082E08093830227
:102EE00081E0809385028FEF809382021092A70287
:102EF000D093A602A9EFB1E0E6E8F2E080E0D813B3
:102F00008DC01092A8028091A802CC0FC82BC0934C
:102F1000A80280918402813009F084C0109284025A
:102F20000E9452086B017C018091A8028093BB0033
:102F300080913A0290913B02A0913C02B0913D02F7
:102F4000892B8A2B8B2BA1F00E94520800913A0208
:102F500010913B0220913C0230913D026C197D0999
:102F60008E099F09061717072807390708F442C07A
:102F70008091BC0083FDD8CF85EC8093BC000E947B
:102F800052086B017C0180918302823009F44CC0AD
:102F9000809182028F3F09F469C080918202803261
:102FA00009F466C080918202803309F463C084E032
:102FB00026C080913A0290913B02A0913C02B091D0
:102FC0003D02892B8A2B8B2B09F483CF0E94520858
:102FD00000913A0210913B0220913C0230913D0257
:102FE0006C197D098E099F090617170728073907ED
:102FF00008F06FCF809139020E94BA1685E01092D6
:10300000FB021092FA021092FD02DF91CF911F9104
:103010000F91FF90EF90DF90CF9008959D91919345
:103020008F5F6DCF85EEA9CF80913A0290913B02E0
:10303000A0913C02B0913D02892B8A2B8B2B09F485
:10304000A2CF0E94520800913A0210913B022091B7
:103050003C0230913D026C197D098E099F090617CB
:1030600017072807390708F08ECFC4CF80E0C7CFF5
:1030700082E0C5CF83E0C3CFEF92FF920F931F93FF
:10308000CF93DF937C01C62F8091D4039091D50319
:10309000009709F459C02091D80331E03093FD0224
:1030A0002093FC021092FB021092FA02DC01ED91D7
:1030B000FC910190F081E02D60E009958701EE24FC
:1030C000E394F12CD1E0C1508091D4039091D503C9
:1030D000CF3F91F1B0E2EB16F104D8F00E94551702
:1030E0008091D4039091D5032091D803D093FD0211
:1030F0002093FC021092FB021092FA02DC01ED9187
:10310000FC910190F081E02D60E00995EE24E394BC
:10311000F12C8091D4039091D503F8016491DC01E6
:10312000ED91FC910190F081E02D0995BFEFEB1A34
:10313000FB0A0F5F1F4FC7CFDF91CF911F910F91F8
:10314000FF90EF900C945517E091E403F091E503A4
:1031500090818091EA038095892380838701C15003
:1031600008F438C0F80184912091D2033091D30340
:10317000232B29F00E947D0C0F5F1F4FF0CF28E01A
:1031800030E040E8E091E003F091E1039091E80342
:10319000582F5423D9F05081952B9083E091E2036E
:1031A000F091E30390815091E903952B9083E09196
:1031B000E203F091E30350819091E9039095952308
:1031C0009083469521503109E9F6D6CF50819095EC
:1031D0009523E3CFDF91CF911F910F91FF90EF9057
:1031E00008951F93CF93DF93EC018D8D9E8D0097F3
:1031F00021F1162F29A131E03093FD022093FC022A
:103200001092FB021092FA02DC01ED91FC91019008
:10321000F081E02D60E009958D8D9E8DDC01ED91B2
:10322000FC910190F081E02D612F09958D8D9E8D8F
:10323000DF91CF911F910C945517ADA5BEA59C9120
:103240008BA9809589238C938B8D9C8D892B31F054
:10325000862FDF91CF911F910C947D0C28E030E0F8
:1032600080E8A9A5BAA599A9462F4823C1F04C9199
:10327000942B9C93ABA5BCA59C914AA9942B9C93A1
:10328000ABA5BCA54C919AA9909594239C93869547
:103290002150310931F7DF91CF911F9108954C9161
:1032A00090959423E6CFDF92EF92FF920F931F93B6
:1032B000CF93DF938091D4039091D503892B09F4A8
:1032C000A5C02091EC033091ED034091EE035091A5
:1032D000EF0360E074E284EF90E00E943F382051F9
:1032E00031094109510956954795379527952093FE
:1032F000B80064E086E09EE00E943C188091BB0329
:103300009091BC038034910509F097C060E287EB8F
:1033100093E00E94F1186091BB03615E87EB93E03C
:103320000E94F1182091BD033091BE03C901079698
:1033300097FD079633E0959587953A95E1F72091AB
:10334000BB033091BC03829F8001839F100D929F2D
:10335000100D1124C091D603D091D7038091D403CE
:103360009091D5030C0F1D1F009709F498C0209170
:10337000D80331E03093FD022093FC021092FB024F
:103380001092FA02DC01ED91FC910190F081E02DA8
:1033900060E40995EE24E394F12CDD24D39480912C
:1033A000D4039091D5030C171D0709F44FC0B0E268
:1033B000EB16F104D8F00E9455178091D403909138
:1033C000D5032091D803D092FD022093FC021092E5
:1033D000FB021092FA02DC01ED91FC910190F08168
:1033E000E02D60E40995EE24E394F12C8091D40360
:1033F0009091D5036991DC01ED91FC910190F081F0
:10340000E02D0995BFEFEB1AFB0AC9CF8091D203DB
:103410009091D303892B31F08091F5039091F603BD
:103420000E94840CE091E603F091E7039081809183
:10343000EB038095892380835CCF60E087EB93E08A
:103440000E94F1186091BB03615068CF0E9455172C
:103450008091D4039091D503892B09F461C0209108
:10346000F0033091F1034091F2035091F30360E0D7
:1034700074E284EF90E00E943F3820513109410905
:10348000510956954795379527952093B800DF91B8
:10349000CF911F910F91FF90EF90DF900895E091F1
:1034A000E403F091E50380819091EA03892B808306
:1034B0000C171D0769F289912091D2033091D30333
:1034C000232B19F00E947D0CF3CF28E030E040E878
:1034D000E091E003F091E1039091E803582F542329
:1034E000D9F05081952B9083E091E203F091E303B2
:1034F00090815091E903952B9083E091E203F09144
:10350000E30350819091E90390959523908346952C
:1035100021503109E9F6CCCF508190959523E3CF26
:10352000E091E603F091E70380819091EB03892B12
:1035300080838091D2039091D303892B09F4A7CF84
:10354000DF91CF911F910F91FF90EF90DF900C943E
:103550006C0C1F93CF93DF93EC01162F8D8D9E8DF6
:10356000892BB1F12DA93EA94FA958AD60E074E2B5
:1035700084EF90E00E943F38205131094109510900
:1035800056954795379527952093B80066EA11110F
:1035900067EACE010E94F1188D8D9E8D892B41F135
:1035A00029AD3AAD4BAD5CAD60E074E284EF90E0E4
:1035B0000E943F38205131094109510956954795DC
:1035C000379527952093B800DF91CF911F910895EB
:1035D0008B8D9C8D892B21F08EAD9FAD0E94840C2C
:1035E000EFA5F8A990818CA9809589238083CECFFF
:1035F000EFA5F8A980819CA9892B80838B8D9C8D58
:10360000892B11F3DF91CF911F910C946C0C90E0FA
:1036100080E00895CF93CFB7F8948091F80181119D
:1036200027C0E4EDFDE08491E8EEFDE09491E82F01
:10363000F0E0EE0FFF1FE455F24FA591B491EC912D
:10364000E92321F461E08AE00E94840761E08AE0D6
:103650000E94B2078CB580618CBD8CB580648CBD36
:1036600061E08DE00E94B20761E08BE00E94B2074A
:103670008091F8018F5F8093F801CFBFCF910895BB
:1036800062E370E080E090E00E9477080E94E90920
:1036900061E08AE00E94B20761E081E00E94B20727
:1036A00061E080E00E94B20760E08AE00E94840747
:1036B00060E080E00E94840760E081E00E9484076F
:1036C00060E081E10E9484079FB7F8948091F8013F
:1036D000882319F081508093F8018091F8018111BD
:1036E00005C08CB58F7B8CBD1092AA029FBF61E094
:1036F0008BE00E94B20761E08DE00E94B20760E0BB
:103700008BE00E94840760E08DE00E9484070E94A5
:103710008F1661E082E10E94B20761E083E10E94BE
:10372000B20760E082E10E94840760E083E10C94CC
:1037300084071092F0020FB6F894A895809160006B
:10374000886180936000109260000FBE0E94401B51
:10375000ECE6F0E080818160808362E370E080E0ED
:1037600090E00E9477088BB387608BBB83B7817F23
:10377000846083BF83B7816083BF889583B78E7F62
:1037800083BF61E080E00E94B20760E080E00E94B9
:103790008407F0E0E0E0099561E086E10E94B2076D
:1037A00060E086E10C9484070F931F93CF93DF931F
:1037B000C8E7D0E001E010E024E030E049E150E06B
:1037C000BE0187EB93E00E942D0B2196CE37D105E9
:1037D00089F7DF91CF911F910F9108950F931F9358
:1037E000CF93DF93C8E7D0E001E010E020E130E0C4
:1037F0004DE050E0BE0187EB93E00E942D0B219637
:10380000CE37D10589F7DF91CF911F910F910895A0
:103810000F931F93CF93DF93C8E7D0E010E000E051
:1038200020E130E04DE050E0BE0187EB93E00E94E4
:103830002D0B2196CE37D10589F7DF91CF911F91BE
:103840000F910895CF93DF938830910508F057C00A
:10385000C62FFC01E25DF34E0C946138361C3E1C11
:103860004F1C5C1C641C661C721C791C70E060E0C0
:1038700085E00E94E30770E060E018C070E060E05F
:1038800085E00E94E30770E060E086E00E94E307C5
:103890006C2F70E089E0DF91CF910C94E30770E02A
:1038A00060E085E00E94E3076C2F70E086E00E94F4
:1038B000E30770E060E0EECF70E060E085E00E943A
:1038C000E307D0E0BE0109C070E0D2CFD0E0BE0176
:1038D00085E00E94E30770E060E086E00E94E30775
:1038E000BE01D8CFD0E0BE0185E00E94E307BE0153
:1038F000DDCFD0E0BE0185E00E94E307E3CFDF919A
:10390000CF910895CF93DF93C091C802D0E0E8EC47
:10391000F2E060E070E0CB019F01285C3240C2170A
:10392000D3078CF0AAE0B0E09B01AC010E94AE3658
:103930006F5F7F4F8F4F9F4F2181620F711D811DE0
:10394000911D3196E9CFDF91CF91089521E0209329
:1039500034014091E6025091E7026091E8027091D3
:10396000E902411551056105710501F18091BE0221
:103970009091BF02A091C002B091C1020196A11D19
:10398000B11D8093BE029093BF02A093C002B0937A
:10399000C10284179507A607B70780F080917000D1
:1039A0008E7F809370002093EF0208951092BE02E4
:1039B0001092BF021092C0021092C102089520918D
:1039C000BD033091BE03C901079697FD079623E01A
:1039D000959587952A95E1F72091BB033091BC031B
:1039E000829FA001839F500D929F500D112470E083
:1039F00060E08091D6039091D7030C94573A0F93CF
:103A00001F930E94DF1C01E010E024E130E04BE056
:103A100050E066E770E087EB93E00E942D0B24E115
:103A200030E04BE050E06FE770E087EB93E00E94FE
:103A30002D0B29E030E04BE050E066E770E087EBCB
:103A400093E00E94760B29E030E04EE150E066E71B
:103A500070E087EB93E00E94760B28E030E04AE0CC
:103A600050E067E770E087EB93E00E94760B28E078
:103A700030E049E050E067E770E087EB93E00E94B8
:103A8000760B8091E4029091E502B0E0A0E04091D5
:103A9000C2025091C3026091C4027091C5028417A2
:103AA0009507A607B70720F41F910F910C94EE1B02
:103AB0000E94081C1F910F910C94D41BCF93DF938D
:103AC000EC0188819981009711F00E9403391982D5
:103AD00018821D821C821B821A82DF91CF91089569
:103AE000FC0180819181009711F00C9403390895B5
:103AF0000E94493AFB0101900020E9F73197AF019C
:103B0000461B570BDC01ED91FC910280F381E02D07
:103B10000994CF93DF93BC018EEF92E00E94B80826
:103B2000EC0165E971E08EEF92E00E947A1D8C0F46
:103B30009D1FDF91CF9108958F929F92AF92BF9278
:103B4000EF92FF920F931F93CF93DF93CDB7DEB722
:103B5000A1970FB6F894DEBF0FBECDBF7C01FA016E
:103B6000CB0119A2223008F42AE08E010F5D1F4F0D
:103B7000822E912CB12CA12CBF01A50194010E9491
:103B80003F38F901CA016A300CF5605DD8016E93C7
:103B90008D01232B242B252B79F790E080E01097C3
:103BA00021F0BD01C7010E947A1DA1960FB6F894BD
:103BB000DEBF0FBECDBFDF91CF911F910F91FF9060
:103BC000EF90BF90AF909F908F900895695CDECF8B
:103BD000AC0170E060E02AE087EB93E00C949C1D60
:103BE0008F929F92AF92BF92CF92DF92EF92FF920D
:103BF000CF93DF936B017C01AC019B010E941238D3
:103C000068E971E0811126C046015701E894B7F8D0
:103C10002FEF3FEF4FE75FE7C501B4010E94123875
:103C200081110CC02FEF3FEF4FE75FE7C501B401F3
:103C30000E9474356CE971E0181664F02FEF3FEFC5
:103C40004FE75FE4C701B6010E940D38181684F4EF
:103C500060EA71E087EB93E0DF91CF91FF90EF9006
:103C6000DF90CF90BF90AF909F908F900C947A1D73
:103C70002FEF3FEF4FE75FECC701B6010E947435AD
:103C800087FDE6CF20E030E0A901C701B6010E9420
:103C90007435D0E0C0E087FF0AC06DE287EB93E0A7
:103CA0000E94AE12EC01F7FAF094F7F8F0942AE0D3
:103CB00037ED43EA5BE3C701B6010E9400374B01D1
:103CC0005C010E94DE376B017C010E9479359B010B
:103CD000AC01C501B4010E94FF364B015C012AE032
:103CE000B701A60187EB93E00E949C1DC80FD91F66
:103CF0006EE287EB93E00E94AE12C80FD91F20E05E
:103D000030E040E251E4C501B4010E94DA354B01D4
:103D10005C010E94DE376B01CB010E94E81DC80FD9
:103D2000D91FB60190E080E00E9479359B01AC017B
:103D3000C501B4010E94FF3620E030E040E251E4CA
:103D40000E94DA350E94DE37CB010E94E81D8C0FFD
:103D50009D1FDF91CF91FF90EF90DF90CF90BF90AC
:103D6000AF909F908F9008950F931F93CF93DF9301
:103D7000EC0188819981009759F02A813B812617AF
:103D8000370730F081E0DF91CF911F910F910895B7
:103D90008B016F5F7F4F0E948C39009759F0998398
:103DA00088831B830A832C813D81232B59F7FC01D7
:103DB0001082E8CF80E0E7CFEF92FF920F931F933E
:103DC000CF93DF93EC017B01198218821B821A8248
:103DD0001D821C82FB0101900020E9F731978F01C1
:103DE000061B170BB8010E94B41E811109C0CE0139
:103DF000DF91CF911F910F91FF90EF900C945E1D7A
:103E00001D830C83B70188819981DF91CF911F9128
:103E10000F91FF90EF900C94723ACF92DF92EF9255
:103E2000FF920F931F93CF93DF9300D000D000D069
:103E3000CDB7DEB70E94821C6B017C010E94FF1C83
:103E400081E08093CB038093CC031092C403109243
:103E5000C3031092C6031092C50389E7C816D104A4
:103E6000E104F10409F471C108F0C2C081E2C8168E
:103E7000D104E104F10408F080C08FE1C816D10438
:103E8000E104F10408F089C18EE0C816D104E10410
:103E9000F10408F061C08BE0C816D104E104F1041C
:103EA00008F032C1D701C6010197A109B10961EC3F
:103EB00072E00697A105B10508F45AC082E080932C
:103EC000CB038093CC038AE090E09093C40380936B
:103ED000C3038FE090E09093C6038093C50384E30F
:103EE000C816D104E104F10409F4A6C208F0CAC15D
:103EF0008DE0C816D104E104F10409F485C208F08C
:103F000073C184E0C816D104E104F10409F488C245
:103F100008F04CC182E0C816D104E104F10409F4B0
:103F200076C208F077C26CE071E0CA94CD28CE2842
:103F3000CF2809F454C10E94531926960FB6F8945D
:103F4000DEBF0FBECDBFDF91CF911F910F91FF90CC
:103F5000EF90DF90CF900895D701C6014597A10952
:103F6000B1096EE871E00497A105B10508F0A6CF8C
:103F700087EB93E00E94B808A1CF84E3C816D10470
:103F8000E104F10409F4CCC0C0F48AE2C816D104FB
:103F9000E104F10409F4BBC083E3C816D104E104D1
:103FA000F10409F4BAC089E2C816D104E104F104AD
:103FB00009F084CF64E872E0DBCF8DE3C816D1044A
:103FC000E104F10408F47ACF81E4C816D104E104D5
:103FD000F10408F4AEC0D701C6018F569109A109BA
:103FE000B10963EA72E00397A105B10508F266CF53
:103FF0008BE9C81681E0D806E104F10409F48AC00F
:10400000D0F587EEC816D104E104F10409F4C2C06A
:10401000C0F483EDC816D104E104F10409F4B4C07E
:104020008DEDC816D104E104F10409F4B0C083E8B1
:10403000C816D104E104F10409F040CF63E972E04D
:1040400097CF87E3C81681E0D806E104F10409F4AC
:10405000A7C081E4C81681E0D806E104F10409F4A0
:10406000A2C081EFC816D104E104F10409F026CF03
:1040700066E471E07DCF83E6C81682E0D806E104ED
:10408000F10409F459C0D8F48FEFC81681E0D806BE
:10409000E104F10409F447C089E0C81682E0D806BB
:1040A000E104F10409F442C085EAC81681E0D806AB
:1040B000E104F10409F002CF63E672E059CF87E72B
:1040C000C81682E0D806E104F104C9F158F46CEE98
:1040D00071E08DE6C81682E0D806E104F10409F427
:1040E00047CFECCE81E8C81682E0D806E104F1049F
:1040F00049F16EEB71E081E6C81684E0D806E10470
:10410000F10409F435CFDACE62EB72E031CF65E726
:1041100072E02ECF64E572E02BCF67E472E028CF27
:104120006AE372E025CF6CE272E022CF6EE172E0CA
:104130001FCF6EE072E01CCF6DEF71E019CF6BED19
:1041400071E016CF6AEC71E013CF0AE010E0109333
:10415000C4030093C30385E090E09093C60380936B
:10416000C5036FEA71E087EB93E00E94B8081093F3
:10417000C4030093C30386E190E09093C603809349
:10418000C5036FE971E0F4CE6CE771E0F1CE6AE649
:1041900071E0EECE68E571E0EBCE69E371E0E8CE68
:1041A00064E271E0E5CE64E171E0E2CE86E0C8163B
:1041B000D104E104F10409F442C108F43AC18BE0EE
:1041C000C816D104E104F10409F40CC165ED70E0F6
:1041D0008CE0C816D104E104F10409F0ACCE87EB01
:1041E00093E00E94B808A7CE8FE1C816D104E1047D
:1041F000F10409F412C118F586E1C816D104E104EE
:10420000F10409F4F8C050F485E1C816D104E104C2
:10421000F10409F090CE64EF70E0E1CF87E1C816B9
:10422000D104E104F10409F4E9C088E1C816D1041D
:10423000E104F10409F07FCE62EE70E0D0CF89E2B4
:10424000C816D104E104F10409F4EDC050F465EAA4
:1042500070E080E2C816D104E104F10409F4BFCF94
:104260006ACE8AE2C816D104E104F10409F4DEC082
:1042700061E870E083E3C816D104E104F10409F4B5
:10428000AECF59CE8DEDC816D104E104F10409F486
:1042900042C008F047C08FE6C816D104E104F1041B
:1042A00009F4A3C0F8F48EE3C816D104E104F104C4
:1042B00009F4A1C040F48DE3C816D104E104F1046F
:1042C00009F4A9CF38CE8FE3C816D104E104F10474
:1042D00009F494C080E4C816D104E104F10409F49F
:1042E000ABCF29CE81E7C816D104E104F10409F46B
:1042F00088C008F47DC065EC70E083E8C816D1047E
:10430000E104F10409F46BCF83EDC816D104E10494
:10431000F10409F010CE8091C6029091C7020E946C
:10432000E81D09CE8BE9C81681E0D806E104F10446
:1043300091F398F581EFC816D104E104F10459F323
:1043400038F487EEC816D104E104F10421F3F3CD6B
:1043500087E3C81681E0D806E104F104E1F281E4C4
:10436000C81681E0D806E104F10409F0E4CDE0913B
:10437000C602F091C70262ED71E0E830F10508F085
:1043800063C0EB53FE4D0C94613822223E223B2247
:10439000442238224122472235228FEFC81681E07D
:1043A000D806E104F10409F4B6CF48F485EAC8164A
:1043B00081E0D806E104F10409F4ADCFBCCD61E79A
:1043C00070E089E0C81682E0D806E104F10409F43F
:1043D00006CF81E6C81684E0D806E104F10409F4AA
:1043E0009ACFA9CD67E071E0FACE60E071E0F7CE38
:1043F0006AEF70E0F4CE6EEE70E0F1CE68EE70E041
:10440000EECE6DED70E0EBCE6FEC70E0E8CE6BEBD6
:1044100070E0E5CE64EB70E0E2CE6BEA70E0DFCEF8
:104420006DE970E0DCCE65E970E0D9CE6DE870E052
:10443000D6CE67E870E0D3CE6BE770E0D0CE68E60A
:1044400070E0CDCE64EA71E0CE0101960E94DC1EE0
:104450004D815E8169817A8187EB93E00E94DC085F
:10446000CE0101960E94701D66CD69EA71E0ECCF25
:104470006FEA71E0E9CF63EB71E0E6CF69EB71E0E1
:10448000E3CF6EEB71E0E0CF66EC71E0DDCF6BEC7B
:1044900071E0DACFEF92FF920F931F93CF93DF93E8
:1044A0008C017B01EB0109900020E9F72197C61BE5
:1044B000D70BBE010E94B41E811109C0C801DF9153
:1044C000CF911F910F91FF90EF900C945E1DF8011A
:1044D000D583C483B70180819181DF91CF911F91F2
:1044E0000F91FF90EF900C94723A85ED8093BC0091
:1044F00080913A0290913B02A0913C02B0913D0222
:104500000796A11DB11D23E0B695A79597958795B0
:104510002A95D1F72091BC0024FD03C0109283029C
:10452000089540913A0250913B0260913C02709193
:104530003D02452B462B472B69F30097A105B1059A
:1045400041F02AE22A95F1F700C00197A109B109CB
:10455000E1CF809139020C94BA16FF920F931F930A
:10456000CF93DF938C01EB01F8800E949836F81608
:1045700021F06F2DC8010E94A036CE01DF91CF91AE
:104580001F910F91FF9008951F93CF93DF931F9278
:10459000CDB7DEB712E01983BE016F5F7F4F90E0A9
:1045A00080E00E94AD221982BE016F5F7F4F81E0E3
:1045B00090E00E94AD228BE08983BE016F5F7F4F48
:1045C00082E090E00E94AD2284E18983BE016F5FAA
:1045D0007F4F83E090E00E94AD221983BE016F5FA0
:1045E0007F4F84E090E00E94AD228AE18983BE0182
:1045F0006F5F7F4F85E090E00E94AD220F90DF91CA
:10460000CF911F9108950F931F93CF93DF9300D005
:10461000CDB7DEB78C017A836983BE016F5F7F4FB0
:104620000E94AD22BE016E5F7F4FC80101960E94BD
:10463000AD220F900F90DF91CF911F910F910895B0
:10464000CF93DF931F92CDB7DEB70E94C42281E0E3
:104650008983BE016F5F7F4F86E090E00E94AD22AC
:1046600065E070E087E090E00E94032364E670E07C
:104670008AE090E00E94032364E670E08CE090E022
:104680000E94032364E670E08EE090E00E94032322
:1046900064E670E080E190E00E94032370E060E057
:1046A00080E290E00E94032389E18983BE016F5F6D
:1046B0007F4F87E190E00E94AD2287E08983BE01B1
:1046C0006F5F7F4F8BE190E00E94AD2260E17EE062
:1046D0008EE190E00E94032361E070E08CE190E0C5
:1046E0000E9403230F90DF91CF9108950C94983688
:1046F0004F925F926F927F928F929F92AF92BF92F2
:10470000CF92DF92EF92FF920F931F93CF93DF939D
:104710006B017C01609102017091030190E080E0E7
:104720000E9479359B01AC01C701B6010E946C372C
:104730000E94DE374B01EB010E94FF1C0091FB033E
:104740001091FC030115110509F44BC069ED71E0EE
:104750008091F7039091F8030E94693A892B09F040
:1047600040C082E08093CB038093CC0384E190E04F
:104770009093C4038093C3031092C6031092C503A1
:1047800066E473E087EB93E00E94B80881E08093D1
:10479000CB038093CC0385E090E09093C403809397
:1047A000C30389E190E09093C6038093C50362E35D
:1047B00073E087EB93E00E94B8080E945319CE0182
:1047C000DF91CF911F910F91FF90EF90DF90CF90ED
:1047D000BF90AF909F908F907F906F905F904F9021
:1047E000089581E08093CB038093CC031092C4039F
:1047F0001092C3031092C6031092C503012B81F0DF
:1048000061EE71E08091F7039091F8030E94693A9C
:10481000892B31F46BE273E087EB93E00E94B808D8
:104820008091FB039091FC03892B81F068EE71E08D
:104830008091F7039091F8030E94693A892B31F433
:1048400065E273E087EB93E00E94B8081092C4031E
:104850001092C3038CE090E09093C6038093C5034D
:1048600086E090E00E947623813009F4C6C008F407
:10487000BDC0823009F4C4C0833009F4C4C081E0F3
:104880008093CB038093CC031092C4031092C30394
:1048900088E190E09093C6038093C50386E090E0A2
:1048A0000E9476238823D1F080E290E00E94762354
:1048B00069EE72E0813071F060EF72E0813050F0AB
:1048C00062EE72E0823031F06BED72E0833011F015
:1048D00064ED72E087EB93E00E94B80886E090E018
:1048E0000E9476238150833008F0F4C080E590E088
:1048F0009093C4038093C3031092C6031092C50320
:1049000020E030E0A901C701B6010E947435882378
:1049100009F4EBC020E030E04AE754E4C701B601F7
:104920000E946C370E94F01D62ED72E087EB93E00D
:104930000E94B8088091D3029091D402892B91F102
:1049400081E08093CB038093CC030FE210E01093BF
:10495000C4030093C30382E090E09093C603809366
:10496000C5036BEC72E087EB93E00E94B80882E02D
:104970008093CB038093CC038091D3029091D40297
:104980008A30910508F0D0C026E330E03093C403AC
:104990002093C3032FE030E03093C6032093C50378
:1049A0000E94E81D20E030E0A901C701B6010E9485
:1049B0007435882309F4BDC082E08093CB038093D3
:1049C000CC038EE590E0CA30D10510F082E590E08E
:1049D0009093C4038093C3038FE090E09093C60349
:1049E0008093C503C4010E94E81DE7CE6EE173E029
:1049F00087EB93E00E94B80842CF68E173E0F8CFFC
:104A000063E173E0F5CF88E190E09093C603809373
:104A1000C50380E290E00E947623813001F158F0D6
:104A2000823089F1833009F441C060E080E290E097
:104A30000E94A03624CF82E08093CB038093CC03E6
:104A40008AE290E09093C4038093C30382E190E0F4
:104A50009093C6038093C5036CE073E0C9CF82E0F6
:104A60008093CB038093CC038AE290E09093C403BD
:104A70008093C30382E190E09093C6038093C503C3
:104A800065E073E0B5CF8093CB038093CC038AE2DB
:104A900090E09093C4038093C30382E190E09093ED
:104AA000C6038093C5036EEF72E0A2CF82E08093CD
:104AB000CB038093CC038AE290E09093C40380936D
:104AC000C30382E190E09093C6038093C50367EF30
:104AD00072E08ECF1092C4031092C30388E190E07D
:104AE0009093C6038093C5030BCF4090DF02509094
:104AF000E0026090E1027090E20220E030E0A90163
:104B0000C301B2010E947435882309F413CF20E059
:104B100030E04AE754E4C301B2010E946C370E94BE
:104B2000F01D60ED72E002CF1093C4030093C30345
:104B300031CF20E030E0A9016091DF027091E00206
:104B40008091E1029091E2020E947435882309F479
:104B500034CE81E08093CB038093CC030AE510E050
:104B60001093C4030093C30382E090E09093C603C4
:104B70008093C50366EC72E087EB93E00E94B8086F
:104B8000609102017091030190E080E00E9479350C
:104B90009B01AC016091DF027091E0028091E10223
:104BA0009091E2020E946C370E94DE37EB0122E016
:104BB0002093CB032093CC036A30710570F421E677
:104BC00030E03093C4032093C3032FE030E03093F0
:104BD000C6032093C503CB0106CF1093C4030093F3
:104BE000C303F3CFCF93882371F087E190E00E9455
:104BF0007623C82F8BE190E00E9476236C2F90E003
:104C0000CF910C94221C60E090E080E0F9CFCF932C
:104C1000C82F8823F1F08091CE029091CF02A0910D
:104C2000D002B091D102892B8A2B8B2B51F40E9498
:104C3000A9086093CE027093CF028093D002909324
:104C4000D10261E080E10E9484078C2FCF910C9407
:104C5000F22560E080E10E9484071092CE0210925B
:104C6000CF021092D0021092D102EFCF1F93CF93B8
:104C7000DF93EC010E947623182FCE0101960E944B
:104C80007623982F812FDF91CF911F9108951F9246
:104C90000F920FB60F9211242F933F938F939F93F0
:104CA000AF93BF938091F2029091F302A091F4022E
:104CB000B091F5023091F10223E0230F2D3758F522
:104CC0000196A11DB11D2093F1028093F2029093F1
:104CD000F302A093F402B093F5028091F602909152
:104CE000F702A091F802B091F9020196A11DB11D41
:104CF0008093F6029093F702A093F802B093F90222
:104D0000BF91AF919F918F913F912F910F900FBEC7
:104D10000F901F90189526E8230F0296A11DB11D34
:104D2000D2CF1F920F920FB60F9211242F933F9361
:104D30004F935F936F937F938F939F93AF93BF93A3
:104D4000EF93FF938EEF92E00E945A09FF91EF914B
:104D5000BF91AF919F918F917F916F915F914F9193
:104D60003F912F910F900FBE0F901F9018951F929B
:104D70000F920FB60F9211242F938F939F93EF935F
:104D8000FF93E0910E03F0910F038081E0911403F3
:104D9000F091150382FD1BC09081809117038F5FF6
:104DA0008F7320911803821741F0E0911703F0E010
:104DB000E250FD4F958F80931703FF91EF919F91E4
:104DC0008F912F910F900FBE0F901F90189580819B
:104DD000F4CF1F920F920FB60F9211242F933F938F
:104DE0004F935F936F937F938F939F93AF93BF93F3
:104DF000EF93FF938091B1029091B2028093B20041
:104E00008091B4029091B502A091B602B091B70220
:104E10000196A11DB11D8093B4029093B502A09399
:104E2000B602B093B7028091B4029091B502A091FE
:104E3000B602B091B7024091AD025091AE026091BE
:104E4000AF027091B00284179507A607B70710F15B
:104E50008091B30281111EC081E08093B3028091E2
:104E6000B4029091B502A091B602B091B702841B32
:104E7000950BA60BB70B8093B4029093B502A09349
:104E8000B602B093B702E091AB02F091AC02099583
:104E90001092B302FF91EF91BF91AF919F918F91CB
:104EA0007F916F915F914F913F912F910F900FBE26
:104EB0000F901F9018951F920F920FB60F9211240A
:104EC0002F933F934F935F936F937F938F939F9312
:104ED000AF93BF93EF93FF938091B900887F8036A3
:104EE00009F44AC0F0F5883209F4A7C018F58031FA
:104EF00009F49BC0B8F4882309F4F9C0883009F498
:104F000094C0FF91EF91BF91AF919F918F917F914D
:104F10006F915F914F913F912F910F900FBE0F9026
:104F20001F901895883109F488C0803251F780931A
:104F3000820214C0803409F49DC040F48033B9F378
:104F40008833F9F68093820285ECB0C0803509F48D
:104F500085C0883509F496C0883499F60E94752278
:104F6000D0CF883909F48CC038F5883729F050F44F
:104F7000883611F0803729F683E0809383021092FF
:104F8000810257C0883809F47BC0803919F0803815
:104F900009F0B7CF80918102803208F071C0E091B2
:104FA000810281E08E0F809381028091BB00F0E04E
:104FB000EF59FD4F80833DC0803B39F0E0F4803AEB
:104FC00009F479C0883A09F09CCF84E08093830289
:104FD0001092600210925F02E091BA02F091BB025F
:104FE000099580915F0281110FC081E080935F027B
:104FF00010923F0209C0803C09F4A6CF883C09F416
:10500000A3CF883B09F07DCFE091600281E08E0F55
:1050100080936002F0E0E15CFD4F80818093BB00F3
:105020009091600280915F0229C08091A8028093D4
:10503000BB0085EC8093BC0064CF9091A702809167
:10504000A602981758F5E091A70281E08E0F809391
:10505000A702F0E0EA57FD4F8081E9CFE091A70277
:1050600081E08E0F8093A7028091BB00F0E0EA57A9
:10507000FD4F80839091A7028091A6029817C8F2F5
:1050800085E8D8CFE091A70281E08E0F8093A70238
:105090008091BB00F0E0EA57FD4F8083809185024C
:1050A00081115CCF81E08093840284EA8093BC000C
:1050B0001092830226CF85EC8093BC00109283026D
:1050C00080918102803230F4E0918102F0E0EF596A
:1050D000FD4F10826091810270E0E091B802F09182
:1050E000B90281E692E00995109281020ACF1092EE
:1050F000820234CF1F920F920FB60F92112410929A
:10510000BE021092BF021092C0021092C1020F9014
:105110000FBE0F901F9018951F920F920FB60F920F
:1051200011242F933F934F935F936F937F938F93AC
:105130009F93AF93BF93EF93FF930E947A28FF91C1
:10514000EF91BF91AF919F918F917F916F915F91FF
:105150004F913F912F910F900FBE0F901F90189578
:105160001F920F920FB60F9211242F933F934F93DC
:105170005F936F937F938F939F93AF93BF93EF93BF
:10518000FF930E947A28FF91EF91BF91AF919F9179
:105190008F917F916F915F914F913F912F910F90E0
:1051A0000FBE0F901F901895CF93DF93EEEFF2E0B4
:1051B0001382128288EE93E0A0E0B0E084839583AE
:1051C000A683B7832FE331E03183208325EC30E0E1
:1051D0003587248724EC30E03787268720EC30E0C1
:1051E000318B208B21EC30E0338B228B22EC30E0B2
:1051F000358B248B26EC30E0378B268B118E128E6C
:10520000138E148ECBEAD3E01B821A828C839D838B
:10521000AE83BF8381E591E09983888367E971E07C
:1052200087EF93E00E94DC1EE7EBF3E0138212822B
:1052300020E830E03583248380E290E09783868302
:105240003187208793878287168A1586148617866A
:10525000168681E0858B848B2FEF3FEF338B228B7B
:10526000318B208B878B108E128E118E8DE691E004
:1052700091838083148E138ED68FC58F10A2178EC4
:105280008FEF84A385A386A387A380A740E85AE174
:1052900066E070E045AB56AB67AB70AF40EA56E8EE
:1052A00061E070E041AF52AF63AF74AF90E596AF8D
:1052B00017AEEBE9F3E023E631E0318320839AE097
:1052C00096878787DF91CF910895CF93DF93CDB7EE
:1052D000DEB7A2970FB6F894DEBF0FBECDBF7894AD
:1052E00084B5826084BD84B5816084BD85B58260EB
:1052F00085BD85B5816085BD80916E00816080939C
:105300006E00109281008091810082608093810004
:105310008091810081608093810080918000816014
:10532000809380008091B10084608093B10080916F
:10533000B00081608093B00080917A008460809397
:105340007A0080917A00826080937A0080917A005E
:10535000816080937A0080917A00806880937A00DF
:105360001092C10085B7806685BF85B7806485BF10
:10537000109268001BBA80916B00816080936B0073
:1053800080916C00816080936C0080916D008460DE
:1053900080936D0080916D00886080936D00809196
:1053A0006D00806180936D0080916D0080688093B6
:1053B0006D008BB387608BBB8091680081608093A8
:1053C0006800809168008260809368008091680026
:1053D00084608093680061E080E00E94B20760E032
:1053E00080E00E9484071092EA021092EB02109271
:1053F000EC021092ED021092EE02E0910E03F09199
:105400000F0382E08083E0910A03F0910B03108286
:10541000E0910C03F0910D0380E18083109216035C
:10542000E0911203F091130386E08083E091100372
:10543000F0911103808180618083E0911003F091ED
:105440001103808188608083E0911003F091110343
:10545000808180688083E0911003F0911103808146
:105460008F7D808381E090E0A0E0B0E08093020334
:1054700090930303A0930403B09305030E94C422F6
:1054800090E080E00E9476238F3F11F40E94202359
:105490001092EF0288EE93E0A0E0B0E08093AD02BE
:1054A0009093AE02A093AF02B093B00286EA9CE163
:1054B0009093AC028093AB02809170008E7F8093BA
:1054C00070008091B0008C7F8093B0008091B1001B
:1054D000877F8093B1008091B6008F7D8093B60066
:1054E000809170008D7F809370008091B100846006
:1054F0008093B1008091B1008C7F8093B10086E0F1
:1055000090E09093B2028093B1021092B402109294
:10551000B5021092B6021092B7021092B3028091B7
:10552000B1029091B2028093B200809170008160CC
:105530008093700064E670E080E090E00E9477085D
:1055400061E080E10E94B20760E080E10E94840790
:1055500064E670E080E090E00E94770861E081E11D
:105560000E94B20761E081E10E94840764E670E076
:1055700080E090E00E94770864E670E080E090E0D0
:105580000E94770861E085E00E94B20761E086E052
:105590000E94B20761E089E00E94B20760E085E006
:1055A0000E94840760E086E00E94840760E086E055
:1055B0000E94840760E089E00E94840761E08FE038
:1055C0000E94B20760E08FE00E9484070E940A1BDD
:1055D0008CB583608CBD8DB58E7F8DBD61E0809173
:1055E000A9030E94B20761E08091A9030E94840789
:1055F0008091AA038F3F09F4BAC060E00E94B2070D
:105600008091AA030E945B07892B09F0B0C061E07A
:105610008091AA030E94B20760E08091AA030E94D1
:10562000840783E090E00197F1F761E08091AA039D
:105630000E94840762E370E080E090E00E947708B7
:1056400040E064E28BE993E00E94EB0C40E066E20C
:105650008BE993E00E94EB0C46E268E48BE993E06F
:105660000E94EB0C40E864E58BE993E00E94EB0CB0
:1056700049EA66E58BE993E00E94EB0C43E068E5BC
:105680008BE993E00E94EB0C48EE6AE58BE993E02E
:105690000E94EB0C40E46AE28BE993E00E94EB0C81
:1056A0004DE362E28BE993E00E94EB0C68E28BE948
:1056B00093E00E94CB0C982F9370933039F0482FD1
:1056C000436068E28BE993E00E94EB0C6CE48BE9A9
:1056D00093E00E94CB0C8077803791F040E76CE438
:1056E0008BE993E00E94800E6CE48BE993E00E94CA
:1056F000CB0C482F40676CE48BE993E00E94EB0CE5
:105700004FEF6EE48BE993E00E94EB0C4FE360E512
:105710008BE993E00E94EB0C4FE362E58BE993E0A9
:105720000E94EB0C6EE68BE993E00E94CB0C182FE5
:1057300065EE78E08EEF92E00E94B808412F50E0CD
:1057400070E060E020E18EEF92E00E949C1D82ED0F
:1057500098E0103959F110F58EEA98E0123131F1E4
:105760008AED98E0183811F181EA98E01FC04FE007
:1057700062E08BE993E00E94EB0C13E062E370E0DF
:1057800080E090E00E94770862E08BE993E00E945D
:10579000CB0C84FF55CF115089F752CF8AEC98E09B
:1057A000113921F082EC98E01239F1F60E94891D3E
:1057B00011501E3F20F08EE598E00E94891D8091D7
:1057C000D6039091D703892B11F10E94DF1C209101
:1057D000BD033091BE038091BB039091BC03213285
:1057E00031050CF0D0C0B9016052710977FF02C0D9
:1057F0006F5F7F4F759567958357910997FD019668
:1058000000E210E023E730E04CE059E0CFC0209107
:10581000BD033091BE03C901079697FD0796B3E01B
:1058200095958795BA95E1F72091BB033091BC031C
:10583000AC01429FC001439F900D529F900D1124D7
:105840000E9467389093D7038093D603892B09F081
:10585000BCCF81E090E09093CA038093C9039093FA
:10586000C8038093C7030E94DF1C1092BE021092EF
:10587000BF021092C0021092C10288E00E945B0732
:10588000892B09F45CC262E0262E312C73E0472E8E
:10589000512C8091F00281110DC081E08093F002C3
:1058A00088E198E20FB6F894A895809360000FBE47
:1058B00090936000A8958EE00E945B076C0185E1E3
:1058C0000E9440081091EF02CD2809F04DC211113D
:1058D0004BC2813092400CF439C26EE182E090E01C
:1058E0000E94221C8091EB029091EC02A091ED02AB
:1058F000B091EE0288519C4FAF4FBF4F8093EB02A7
:105900009093EC02A093ED02B093EE0281369A4E92
:10591000A105B105B8F080916C008E7F80936C007A
:105920000E94E90961E080E00E94B2078EE00E94D7
:105930005B07892BD9F360E080E00E94840781E057
:105940008093EF028091EA0281110AC00E94401BFD
:1059500081E08093EA02809170008E7F80937000D6
:1059600068EE73E080E090E00E94770880E090E0CD
:10597000892B09F48ECF0E944609882309F489CF28
:105980000E94000086CFB9016054710977FF02C000
:105990006F5F7F4F759567958255910997FD0196C9
:1059A00000E410E022E530E04CEE5AE09595879552
:1059B0000E945A1582E08093D9038091D40390917C
:1059C000D503892B09F4DFC08CE38093D8031092B0
:1059D000BD021092BC021092FB021092FA020E94C9
:1059E0009C1685EB98E09093BB028093BA0286EBFD
:1059F00098E09093B9028093B8028091DF0387FD0D
:105A00001EC061E00E94B20761E08091DF030E9446
:105A1000840761E070E080E090E00E94770860E039
:105A20008091DF030E9484076AE070E080E090E0EC
:105A30000E94770861E08091DF030E9484078091D3
:105A4000D4039091D503892B09F42AC12091EC034A
:105A50003091ED034091EE035091EF0360E074E26A
:105A600084EF90E00E943F382051310941095109EB
:105A700056954795379527952093B80064E088E0C0
:105A800099E00E943C186091BD03615087EB93E060
:105A90000E94F11864E084E099E00E943C18809133
:105AA000D90360E1813009F064E187EB93E00E9463
:105AB000F11864E080E099E00E943C188FE8809340
:105AC000F4038091BB039091BC038038910509F0E9
:105AD000FEC08091BD039091BE038034910509F012
:105AE00006C18091D903813009F014C18FE98093F8
:105AF000F40312E16AED87EB93E00E94F118612F45
:105B000087EB93E00E94F11861E887EB93E00E9435
:105B1000F1186091F40387EB93E00E94F11869EDAE
:105B200087EB93E00E94F1188091D90362E2813003
:105B300009F061EF87EB93E00E94F11866E08AEFCD
:105B400098E00E943C188091D4039091D503892B52
:105B500009F4E2C02091F0033091F1034091F20387
:105B60005091F30360E074E284EF90E00E943F38CC
:105B70002051310941095109569547953795279587
:105B80002093B80066CE61E08091DD030E94B207E9
:105B900061E08091DE030E94B2078091DD03082E50
:105BA000000C990BFC01E653F24FE491F0E0EE0F8C
:105BB000FF1FEA54F24F259134913093E50320936F
:105BC000E403FC01E252F24FE491E093EA03809196
:105BD000DE03082E000C990BFC01E653F24FE49112
:105BE000F0E0EE0FFF1FEA54F24FA591B491B0938D
:105BF000E703A093E603FC01E252F24FE491E09345
:105C0000EB038C91E82BEC938091D2039091D3031A
:105C1000892B19F00E940A1BF0CE61E08091DB0312
:105C20000E94B20761E08091DC030E94B20780917C
:105C3000DB03082E000C990BFC01E653F24FE491B4
:105C4000F0E0EE0FFF1FEA54F24F259134913093AC
:105C5000E1032093E003FC01E252F24FE491E09370
:105C6000E8038091DC03082E000C990BFC01E6533D
:105C7000F24FE491F0E0EE0FFF1FEA54F24FA591CE
:105C8000B491B093E303A093E203FC01E252F24F1C
:105C9000E491E093E9038C91E095E823EC93ADCE99
:105CA0008091D2039091D303892B31F08091F50339
:105CB0009091F6030E94840CE091E603F091E703D3
:105CC00090818091EB03809589238083D7CE8036A5
:105CD000910589F48091BD039091BE03409739F4FA
:105CE0008091D903813029F480E18093F40312E09C
:105CF00001CF8FEAFACF80349105C9F78091BD03B7
:105D00009091BE03809799F78091D903813011F467
:105D100080E1EDCE8FECEBCEE091E603F091E7036E
:105D200080819091EB03892B80838091D2039091A5
:105D3000D303892B09F48DCD0E946C0C8ACD64E1CC
:105D400070E080E090E00E94770897CD1092EB021F
:105D50001092EC021092ED021092EE026EE181E0E0
:105D600090E00E94221CEECD8CE190E00E94762310
:105D7000FCE38F9FC0011124092E000CAA0BBB0B62
:105D80008093E6029093E702A093E802B093E902C1
:105D90008EE190E00E9436269093E5028093E40223
:105DA000112339F06EE190E080E00E94221C0E94F5
:105DB000991B8091EA02882319F0F0E0E0E0099550
:105DC00080913401882379F0109234018091000190
:105DD000909101010196181619060CF461C0909378
:105DE00001018093000104E011E044E3642E41E0EE
:105DF000742EFF24F39488248394912CF80112824A
:105E000013821186108682850E945B07892B09F018
:105E1000FFC00E94A908F80120813181213031059D
:105E200009F4B7C008F4ABC02230310509F4C5C08D
:105E30002330310509F4D4C0045F1F4F601671068A
:105E4000E9F6809024019090250120913001309155
:105E50003101821A930A80910701882341F081E081
:105E60008093E3020E940D1F80E00E94F225809142
:105E7000E302882309F45CC31091060180911201AA
:105E8000882309F4D0C082E00E945B07892B09F0C7
:105E9000C3C064E170E080E090E00E947708F3CF37
:105EA000109201011092000161E08FE00E948407CE
:105EB0006AE070E080E090E00E94770810E2812CB8
:105EC000912C540184E10E944008092E000CAA0B79
:105ED000BB0B880E991EAA1EBB1E115099F760E0DD
:105EE0008FE00E948407C501B4010E94793520E04B
:105EF00030E04AE754E40E94DA352CE83EE24AEB0F
:105F00005FE30E94DA3520E030E040E450E40E9494
:105F1000DA3520E030E040E058E30E94DA350E94B4
:105F2000DE376093C2027093C3028093C4029093E1
:105F3000C50260387C408105910510F40E94991BD0
:105F40000E94081C8091E4029091E502B0E0A0E07C
:105F50004091C2025091C3026091C4027091C50287
:105F600084179507A607B70728F40E94EE1B0E9426
:105F7000531939CF0E94081C0E94D41BF8CF0E94ED
:105F8000A908F80164837583868397839182808250
:105F900053CFA480B580C680D7806A197B098C094D
:105FA0009D096F3171058105910508F445CFF28295
:105FB00031872087318220823FCF248135814681FD
:105FC0005781621B730B840B950B693E73408105EF
:105FD000910508F431CFF801F382518240822CCF31
:105FE0002481358146815781621B730B840B950B8D
:105FF0006F3171058105910508F41ECF0E94A90833
:10600000F80164837583868397839186808614CF95
:10601000F8011182108210CF8091C802882351F1BB
:1060200081508093C802112309F493C10E94821CFD
:106030006037710509F4D3C00CF069C0693271058D
:1060400009F4EAC05CF51091C8026731710509F4E2
:1060500037C1B4F46531710509F413C18CE090E0E7
:106060006631710509F40FC18091C8028F5F80937A
:10607000C802E6C01092E30280E00E94F22576CCCE
:106080006F31710509F445C16032710509F447C1EA
:106090006831710549F780E190E0F5C06E33710514
:1060A00009F44EC1A4F46333710509F4D7C06D330C
:1060B000710509F440C16A327105B1F68091C202DE
:1060C0009091C3029093C7028093C602CDCF6034F3
:1060D000710509F43BC10CF436C16F36710521F628
:1060E0001982BE016F5F7F4F86E090E00E94AD2273
:1060F0001092C8021092C9021092CA021092CB02EA
:106100001092CC021092CD021092E30299C0613F2E
:10611000710509F4EBC084F56338710509F479C0A1
:1061200064F46137710509F471C06937710509F0CC
:106130009BCF8091C80281509ACF6D3D710509F4C3
:10614000ACC0673E710509F4BEC0633D710509F03E
:106150008BCF8091C6029091C702892B31F481E0E8
:1061600090E09093C7028093C6026091C60270913E
:10617000C7028AE090E047C0653AF1E07F0709F482
:1061800057C0CCF4613431E0730709F4CBC06B39EC
:1061900041E0740709F443C06733714009F064CFEC
:1061A0008091C6028983BE016F5F7F4F87E190E0D7
:1061B0000E94AD22BECF6930E2E07E0709F451C0F3
:1061C0006136F4E07F0781F06F3F714009F04CCFFA
:1061D0006091C6027091C7028CE190E026C087E012
:1061E00090E00E9436266ECF81E08983BE016F5F0A
:1061F0007F4F86E090E00E94AD226091C6027091D0
:10620000C70287E090E00E94032372CF82E0898377
:1062100068CF0E9420238DCF8EE190E0E2CF609185
:10622000C6027091C7028EE190E00E94032381CFE5
:106230008091C2029091C3029093C7028093C602DC
:1062400080910E010E945B07892B09F082C064E1F6
:1062500070E080E090E00E947708F2CF8CE190E05F
:10626000C0CF80910E010E945B07892B39F46AE050
:1062700070E080E090E00E947708F3CF0E94991BC5
:1062800058CF8AE090E00E9436269093C702809310
:10629000C6021F5F1093C802D3CF8091C6029091AF
:1062A000C702892B31F481E090E09093C70280937C
:1062B000C6026091C6027091C7028CE090E0A3CF45
:1062C0008EE090E0E0CF8091C6029091C702892BCA
:1062D00031F481E090E09093C7028093C602609110
:1062E000C6027091C7028EE090E08DCF8091C60209
:1062F0009091C702892B31F481E090E09093C7021E
:106300008093C6026091C6027091C70280E190E05E
:106310007ACF87E190E00E94762390E0B6CF8BE1C0
:1063200090E0F9CF8091C6028983BE016F5F7F4FF5
:106330008BE190E03DCF70E060E080E290E063CFE1
:1063400061E070E0FACF62E070E0F7CF63E070E008
:10635000F4CF8114910409F4C3C0E091C802F0E0C5
:10636000E653FD4FCF01885C9240069710F41192DE
:10637000F9CF0E94821C613471058105910508F0F6
:1063800045C06D3371058105910508F0ACC06931D8
:10639000710581059105E8F4653171058105910567
:1063A00008F0A1C0613071058105910538F16730B1
:1063B00071058105910508F4B8C06B507109810918
:1063C00091096330710581059105C0F463E070E0C7
:1063D00079C06B3271058105910598F469327105B8
:1063E0008105910508F06CC06F517109810991090F
:1063F000623071058105910508F462C061E070E0CA
:1064000061C06353710981099109F2CF613F710540
:1064100081059105B1F000F5633D71058105910598
:1064200081F028F46F56710981099109CACF6D3D39
:1064300071058105910529F0673E7105810591057A
:10644000E9F68091C6029091C7028F5E984D880D43
:10645000991D61E177E266C06B3931E07307810510
:10646000910509F443C0A8F4673351E0750781052D
:106470009105D9F0613471408105910509F0BECFD5
:106480008091C6029091C702880D991D8770992747
:106490003BC06F3FF1E07F0781059105D1F1613687
:1064A00074408105910509F0A9CF8091C6029091B1
:1064B000C7028B599F4F880D991D65E670E032C069
:1064C00062E070E0E091C802F0E0E753FD4F8081A8
:1064D000860F972F911D880D991D0E942B38808360
:1064E0000E940D1F43CA64E070E0ECCF8091C602A9
:1064F0009091C70288519C4F880D991D68EE73E0FA
:106500000E9417388854944F9093C7028093C60214
:1065100075CF8091C6029091C702CC96880D991DC7
:106520006CE370E00E941738EFCF66E070E0CACFEE
:1065300086E090E00E9476238114910409F064C003
:1065400088A388A1813041F487E090E00E9436263C
:106550009093D4028093D3026EEE71E087EF93E0C4
:106560000E944A2288E00E945B07892B09F06CC0D8
:106570008091FB039091FC03892B59F069ED71E048
:106580008091F7039091F8030E94693A892B09F4EE
:106590005BC08091D202811157C088A1813009F47B
:1065A00099C008F470C0823009F4EDC088E00E9400
:1065B0005B07892B09F4DAC988A1813009F4D6C9AF
:1065C0008BE993E00E94940E882309F4CFC98BE9EC
:1065D00093E00E94060A882309F4C8C94EE953E0F3
:1065E0005AA349A385ED882E82E0982E9DED692E51
:1065F00092E0792EF401DA019D91819198135DC1A9
:106600006E167F06C9F7B2C9880D992D911D0396A4
:10661000B2010E942B3888A3BE01605E7F4F86E0E6
:1066200090E00E94AD221092DF021092E0021092E0
:10663000E1021092E2021092D5021092D40210925E
:10664000D3021092D2027DCF63EF71E087EF93E027
:106650000E944A2280E00E94072668EE71E087EFE0
:1066600093E00E944A2280E290E00E9476238230EA
:1066700009F400C1833009F400C1813009F0E4C09D
:106680008CE090E0E3C081E00E940726A8950E947C
:10669000A9080091CE021091CF022091D002309132
:1066A000D102601B710B820B930B0E9479356093B2
:1066B000DF027093E0028093E1029093E2020E9475
:1066C000782388E00E945B07892BE9F280E00E9432
:1066D00007266CCF20910201309103018091D302F3
:1066E0009091D402289FB001299F700D389F700DA2
:1066F000112490E080E00E9479354B015C0120E09C
:1067000030E64AEE57E40E940D3818163CF4812C0E
:1067100030E8932E3BE3A32E36E4B32E81E00E94B3
:106720000726A8950E94A9080091CE021091CF02D9
:106730002091D0023091D102601B710B820B930B20
:106740000E9479356093DF027093E0028093E1024A
:106750009093E2020E947823A50194016091DF02E8
:106760007091E0028091E1029091E2020E940D3866
:1067700087FDD7CF80E00E94072688E00E945B0754
:10678000892BD9F313CF0091D3021091D4028091B9
:10679000020190910301089FB001099F700D189F9D
:1067A000700D112490E080E00E9479354B015C016E
:1067B00020E030E64AEE57E40E940D3818163CF40B
:1067C000812C20E8922E2BE3A22E26E4B22E012B60
:1067D00009F4ECCE81E00E940726A8950E94A90842
:1067E0000091CE021091CF022091D0023091D102BF
:1067F000601B710B820B930B0E9479356093DF0253
:106800007093E0028093E1029093E2020E94782369
:106810002091D3023091D4028217930770F4A5011E
:1068200094016091DF027091E0028091E102909109
:10683000E2020E940D3887FDD0CF80E00E9407263B
:1068400081E08093D202B2CE8AE090E00E943626A8
:1068500090930301809302011092DF021092E002F4
:106860001092E1021092E20260E070E0CB010E941F
:1068700078239CCE8EE090E0E9CF80E190E0E6CFF7
:106880000FEF1FEF5AC00E945E1D75C00E940339B2
:106890008B899C899A8F898F8D899E899C8F8B8FFC
:1068A0008F89988D9E8F8D8F1C8A1B8A1E8A1D8AC8
:1068B00081C060E070E0CB018AC082E18F8F80E30D
:1068C000898387E08A839E012D5F3F4F42E0BE01AE
:1068D0006F5F7F4F8BE993E00E940A0D811146C8DC
:1068E000AA24A394C12CF12CE12C8E01015E1F4F30
:1068F0009E012F5F3F4F44E0B9018BE993E00E9476
:10690000610D811133C8BE016D5F7F4FCE01499685
:106910000E94DC1E8D8D9E8D892B09F4B1CF098DCF
:106920001A8D6EEF7FEFC8010E945E3A009709F45E
:10693000A7CFFC01E01BF10B8F0167E971E0CE01ED
:1069400043960E94DC1E8D8D9E8D0097D1F080179E
:10695000910708F48C01E98DFA8DE00FF11FF080AA
:106960001082698D7A8DCE0143966115710509F407
:106970008ACF0E944A22898D9A8D080F191FF8012B
:10698000F082898D9A8D009709F482CF6B897C897A
:106990006115710509F47ACF4B8D5C8D2F89388D87
:1069A0004217530708F472CF0E94723A8F89988D6C
:1069B0009E8F8D8F188E1F8ACE0143960E94701D68
:1069C000898D9A8D009709F474CF0E9438357093A1
:1069D000D4026093D302E9A1FAA18191FAA3E9A3B9
:1069E000F40181934F016E167F06A9F780E58B8B2A
:1069F0001C8A9E012B5E3F4F42E0BE016D5E7F4FC1
:106A00008BE993E00E940A0D811110C0A12CC12CCA
:106A1000F12CE12C10E000E030E020E044E0BE0189
:106A20006D5E7F4F8BE993E00E94610D1092D20260
:106A30001092DF021092E0021092E1021092E20244
:106A4000CE0149960E94701D0C94B62C8DE691E003
:106A50009093B8038093B7038091D6039091D703A6
:106A6000009711F00E94033987EF93E00C94701D9A
:106A70001F93FC0199278827BC01E89411911032DB
:106A8000E9F3193010F01E30C8F31B3251F01D32FB
:106A900049F4689406C00E945F35610F711D811D25
:106AA000911D119110531A30B0F33EF490958095DA
:106AB000709561957F4F8F4F9F4F1F910895592F6C
:106AC000482F372F262F660F771F881F991F660FB5
:106AD000771F881F991F620F731F841F951F660FF2
:106AE000771F881F991F08950E94B63508F481E02A
:106AF0000895E89409C097FB3EF4909580957095B1
:106B000061957F4F8F4F9F4F9923A9F0F92F96E9F9
:106B1000BB279395F695879577956795B795F1116E
:106B2000F8CFFAF4BB0F11F460FF1BC06F5F7F4F0B
:106B30008F4F9F4F16C0882311F096E911C077231D
:106B400021F09EE8872F762F05C0662371F096E826
:106B5000862F70E060E02AF09A95660F771F881FF5
:106B6000DAF7880F9695879597F90895990F000899
:106B7000550FAA0BE0E8FEEF16161706E807F9070F
:106B8000C0F012161306E407F50798F0621B730BAA
:106B9000840B950B39F40A2661F0232B242B252B2B
:106BA00021F408950A2609F4A140A6958FEF811DCE
:106BB000811D08950E94ED350C945E360E9450367A
:106BC00038F00E94573620F0952311F00C94473688
:106BD0000C944D3611240C9492360E946F3670F34B
:106BE000959FC1F3950F50E0551F629FF001729F72
:106BF000BB27F00DB11D639FAA27F00DB11DAA1F81
:106C0000649F6627B00DA11D661F829F2227B00DCD
:106C1000A11D621F739FB00DA11D621F839FA00D58
:106C2000611D221F749F3327A00D611D231F849FA8
:106C3000600D211D822F762F6A2F11249F575040FF
:106C40009AF0F1F088234AF0EE0FFF1FBB1F661F7A
:106C5000771F881F91505040A9F79E3F510580F043
:106C60000C9447360C9492365F3FE4F3983ED4F38D
:106C7000869577956795B795F795E7959F5FC1F7E7
:106C8000FE2B880F911D9695879597F9089597F992
:106C90009F6780E870E060E008959FEF80EC0895C2
:106CA00000240A94161617061806090608950024EB
:106CB0000A9412161306140605060895092E039465
:106CC000000C11F4882352F0BB0F40F4BF2B11F4D9
:106CD00060FF04C06F5F7F4F8F4F9F4F089557FD38
:106CE0009058440F551F59F05F3F71F04795880F3A
:106CF00097FB991F61F09F3F79F0879508951216D1
:106D000013061406551FF2CF4695F1DF08C016167C
:106D100017061806991FF1CF86957105610508942D
:106D20000895E894BB2766277727CB0197F9089544
:106D3000F999FECF92BD81BDF89A992780B5089543
:106D4000262FF999FECF1FBA92BD81BD20BD0FB687
:106D5000F894FA9AF99A0FBE019608950E94F036B7
:106D6000A59F900DB49F900DA49F800D911D11249F
:106D700008952F923F924F925F926F927F928F92DF
:106D80009F92AF92BF92CF92DF92EF92FF920F93BA
:106D90001F93CF93DF93CDB7DEB7CA1BDB0B0FB6C4
:106DA000F894DEBF0FBECDBF09942A883988488881
:106DB0005F846E847D848C849B84AA84B984C88417
:106DC000DF80EE80FD800C811B81AA81B981CE0F0E
:106DD000D11D0FB6F894DEBF0FBECDBFED010895F3
:106DE000A29FB001B39FC001A39F700D811D11240C
:106DF000911DB29F700D811D1124911D0895505851
:106E0000BB27AA270E9417370C945E360E94503683
:106E100038F00E94573620F039F49F3F19F426F4D9
:106E20000C944D360EF4E095E7FB0C944736E92FB1
:106E30000E946F3658F3BA176207730784079507E5
:106E400020F079F4A6F50C9491360EF4E0950B2E13
:106E5000BA2FA02D0B01B90190010C01CA01A001AC
:106E60001124FF27591B99F0593F50F4503E68F107
:106E70001A16F040A22F232F342F4427585FF3CF48
:106E8000469537952795A795F0405395C9F77EF419
:106E90001F16BA0B620B730B840BBAF09150A1F062
:106EA000FF0FBB1F661F771F881FC2F70EC0BA0FE8
:106EB000621F731F841F48F4879577956795B79570
:106EC000F7959E3F08F0B0CF9395880F08F099276B
:106ED000EE0F9795879508950E9480370C945E3643
:106EE0000E94573658F00E94503640F029F45F3F18
:106EF00029F00C94473651110C9492360C944D366F
:106F00000E946F3668F39923B1F3552391F3951BD3
:106F1000550BBB27AA2762177307840738F09F5FBA
:106F20005F4F220F331F441FAA1FA9F335D00E2E27
:106F30003AF0E0E832D091505040E695001CCAF794
:106F40002BD0FE2F29D0660F771F881FBB1F261757
:106F500037074807AB07B0E809F0BB0B802DBF012E
:106F6000FF2793585F4F3AF09E3F510578F00C94FD
:106F700047360C9492365F3FE4F3983ED4F38695FF
:106F800077956795B795F7959F5FC9F7880F911D1E
:106F90009695879597F90895E1E0660F771F881F0A
:106FA000BB1F621773078407BA0720F0621B730BBD
:106FB000840BBA0BEE1F88F7E09508950E94773690
:106FC00088F09F5798F0B92F9927B751B0F0E1F0AA
:106FD000660F771F881F991F1AF0BA95C9F714C05A
:106FE000B13091F00E949136B1E008950C94913641
:106FF000672F782F8827B85F39F0B93FCCF3869593
:1070000077956795B395D9F73EF4909580957095EF
:1070100061957F4F8F4F9F4F08950E94B63508F4BA
:107020008FEF08950E94B635880B990B0895AA1B1F
:10703000BB1B51E107C0AA1FBB1FA617B70710F063
:10704000A61BB70B881F991F5A95A9F78095909595
:10705000BC01CD01089597FB072E16F4009407D0CC
:1070600077FD09D00E94173807FC05D03EF49095B3
:1070700081959F4F0895709561957F4F0895A1E286
:107080001A2EAA1BBB1BFD010DC0AA1FBB1FEE1FA2
:10709000FF1FA217B307E407F50720F0A21BB30BED
:1070A000E40BF50B661F771F881F991F1A9469F769
:1070B00060957095809590959B01AC01BD01CF01C5
:1070C0000895EE0FFF1F0590F491E02D09940F93A2
:1070D0001F93CF93DF938230910510F482E090E00C
:1070E000E091FF03F091000430E020E0B0E0A0E088
:1070F000309799F42115310509F44AC0281B390B42
:1071000024303105D8F58A819B816115710589F19B
:10711000FB0193838283FE0111C040815181028172
:10712000138148175907E0F04817590799F4109749
:1071300061F012960C93129713961C933296CF011E
:10714000DF91CF911F910F9108950093FF0310934A
:107150000004F4CF2115310551F04217530738F0E0
:10716000A901DB019A01BD01DF01F801C1CFEF01E7
:10717000F9CF909300048093FF03CDCFFE01E20F7F
:10718000F31F819391932250310939832883D7CFFC
:107190002091FD033091FE03232B41F42091370110
:1071A000309138013093FE032093FD032091350187
:1071B000309136012115310541F42DB73EB740918C
:1071C000390150913A01241B350BE091FD03F091F8
:1071D000FE03E217F307A0F42E1B3F0B2817390715
:1071E00078F0AC014E5F5F4F2417350748F04E0F23
:1071F0005F1F5093FE034093FD03819391939FCFB4
:10720000F0E0E0E09CCFCF93DF930097E9F0FC0142
:10721000329713821282A091FF03B0910004ED0116
:1072200030E020E01097A1F420813181820F931F7C
:107230002091FD033091FE032817390709F061C042
:10724000F093FE03E093FD03DF91CF910895EA01EF
:10725000CE17DF07E8F54A815B819E014115510594
:10726000B1F7E901FB83EA8349915991C40FD51F16
:10727000EC17FD0761F4808191810296840F951FC0
:10728000E90199838883828193819B838A83F0E0DB
:10729000E0E012968D919C9113970097B9F52D918E
:1072A0003C911197CD010296820F931F2091FD030F
:1072B0003091FE032817390739F6309751F51092AF
:1072C00000041092FF03B093FE03A093FD03BCCF14
:1072D000D383C28340815181840F951FC817D9077A
:1072E00061F44E5F5F4F88819981480F591F518328
:1072F00040838A819B81938382832115310509F024
:10730000B0CFF0930004E093FF039ECFFD01DC01BA
:10731000C0CF13821282D7CFB0E0A0E0E2E9F9E358
:107320000C94BB368C01009751F4CB010E94673856
:107330008C01C801CDB7DEB7E0E10C94D736FC0173
:10734000E60FF71F9C0122503109E217F30708F4FA
:107350009DC0D901CD91DC911197C617D70798F040
:10736000C530D10530F3CE0104978617970708F38F
:10737000C61BD70B2297C193D1936D937C93CF01FA
:107380000E940339D6CF5B01AC1ABD0A4C018C0EAA
:107390009D1EA091FF03B0910004512C412CF12CB3
:1073A000E12C109731F58091FD039091FE03881533
:1073B000990509F05CC04616570608F058C0809140
:1073C000350190913601009741F48DB79EB74091F9
:1073D000390150913A01841B950BE817F90708F021
:1073E00055C0F093FE03E093FD03F90171836083C0
:1073F000A0CF8D919C91119712966C901297139635
:107400007C901397A815B90559F56C0142E0C40E9C
:10741000D11CCA14DB0420F1AC014A195B09DA0162
:107420001296159780F06282738251834083D9014E
:107430006D937C93E114F10471F0D7011396FC93E2
:10744000EE93129776CF22968C0F9D1FF9019183B0
:107450008083F301EFCFF0930004E093FF0369CF43
:107460004816590608F42C017D01D3019ACFCB01AF
:107470000E9467387C01009749F0AE01B8010E9474
:107480004E3AC8010E940339870153CF10E000E053
:1074900050CF81E090E0F8940C94793AFB01DC0144
:1074A00002C001900D9241505040D8F70895DC0180
:1074B00001C06D9341505040E0F70895FC01819167
:1074C000861721F08823D9F7992708953197CF019E
:1074D0000895FB01DC018D91019080190110D9F311
:1074E000990B0895FB01DC0101900D920020E1F75A
:1074F000089517E0C6E0D7E004C0FE010E9461389D
:0C7500002196C730D107C9F7F894FFCFDF
:10750C0001000A000000000000000000000007005D
:10751C00000000000000000000000200000000005D
:10752C00000000000000040000000000000000004B
:10753C000000030001000001048000000000007C3A
:10754C0009DC080909C9093A0918092C09000000C5
:10755C00002617F916071B3107F216DF16D0160096
:10756C00000000F20E940E060A00000000AE12DCC1
:10757C0008071BB708BD0B310753152B1547153BD7
:10758C0015BB1531077410A91A2D0B760B741457F3
:10759C0014DF1380130D0A006E616E00696E6600B5
:1075AC006F7666004E6F6E650057686974650052A1
:1075BC00656400477265656E00426C7565004D61CF
:1075CC0067656E7461004379616E0059656C6C6F10
:1075DC007700556E6B6E6F77004E6F7468696E67CF
:1075EC00004C697175696400536F6C6964004348A1
:0875FC00413000434841320018
:00000001FF
